:020000040000FA
:100000000C9462190C948A190C948A190C94452E3C
:100010000C948A190C948A190C948A190C948A19D4
:100020000C948A190C948A190C948A190C948A19C4
:100030000C948A190C948A190C948A190C948A19B4
:100040000C94FB2D0C948A190C94C92D0C94A32D9F
:100050000C948A190C941C2F0C948A190C948A19EC
:100060000C948A190C948A1900000000000F1DC21C
:100070000800054442080003845FBF000FE44410F9
:10008000000115451000054CC97F8009244F9000E0
:1000900007C4C11000054D413F00055443810007CE
:1000A000C44D02000544411400055541080007C82D
:1000B0008104000000000000000000000001083F73
:1000C000FE001FFF810000004002000007FE0FF845
:1000D000000402080800040208880007FE088800DF
:1000E0000402088800040208880007FE088800044B
:1000F00002094800040202300007FE040C0004025A
:1001000018040000000000000000000000011000C2
:1001100080001FFF80800001103FFF0000400408A6
:100120000007FC040800044404100004440210000A
:1001300004440220001FFF812000004000C0000096
:10014000A00130000110020800060C0C0700180383
:10015000B0020000000000000000000000004000AD
:10016000800000400080000FFF3FFF0008410408AE
:100170000008410408000841041000084102100072
:100180000FFF0220000841012000004000C00000D5
:1001900040013000004002080000400C0700004011
:1001A000300200000000000000000000001FDF100F
:1001B000200002120C20000224042000047F802072
:1001C000000424B820000FA488500014BF885000F9
:1001D00004A488500004A488480004BF8888000450
:1001E000A48A880007A48C84000444890700008145
:1001F000860200000000000000000000000FF00474
:1002000091000440025200047F905400045088FF83
:100210000007D08481000451008100044901FF00DF
:1002200007CA0281000444048100044A1CFF00073D
:10023000EA0481000C510481000061C48500004083
:100240008082000000000000000000000007FF8026
:100250002000008407FF00008404010000840401E2
:100260000000840401000FFFC7FF000084040000A9
:100270000084040000008405FF00008405010001E3
:10028000040901000104090100020411FF00040433
:1002900001010000000000000000000000008204D6
:1002A000FF00004402010007FF9021000010102110
:1002B00000001017FD0000101021000FFFD061009A
:1002C000001010A1000028112100002812210000B8
:1002D00044142100008210A1000301D045000C004D
:1002E0009002000000000000000000000008441020
:1002F000FE00042810920005FF22920000103C929C
:100300000000100892001CFE109200041020FE0055
:1003100004103E920005FF80920004100092000538
:10032000100E92000610309200041000FE00001023
:100330000082000000000000000000000007DF88CD
:1003400040000A24104000114210FE0004002282E6
:100350000002FF3D020008010A420009F9103200C4
:10036000090920120009F93E0200090900020009EA
:10037000090E020009F930220008050014000802E5
:10038000000800000000000000000000000FC3F1A2
:10039000E0000FE3F1F8000C70C19E000C30C18644
:1003A000000C30C183000C30C183000C60C183009D
:1003B0000C60C183000FC0C183000FC0C186000C58
:1003C00000C186000C00C198000C03F1F8000C037A
:1003D000F1E0000000000000000000000000200824
:1003E00020000FFF09FC00002008000000203E88CC
:1003F0000003FE08500002020BFE0003FE0C40004A
:10040000020218400003FE2BFE000202084800030F
:10041000FE088800020208500002022830001FFF78
:1004200091CC0000000000000104047C000088045E
:1004300044000FFF3F4400002004440000200C440F
:100440000000200E44001FFF9544000020144400CB
:10045000005024440000500444000088044500017A
:100460000404850006038503001801040000000051
:1004700000000000000000000000000000047E21D9
:10048000FC0004421104001F7E090400044221FC08
:10049000000542110400067E1104000C0005FC005A
:1004A00015FF880000040813FE00044832520004BF
:1004B0004F125200044812520014A8125200091F91
:1004C00097FF000000000000000000000002103D47
:1004D000FC000210250400041025040005FFBDFCEB
:1004E000000C102520000C38252000143825FE00B3
:1004F00004543D20000454251000049225100005EA
:1005000011A5090006113D450004102583000410C3
:10051000010100000000000000000000001FC810E2
:100520002000124A0C20001AC9042000174800209D
:10053000001FFFB8200002080850001FC808500024
:10054000020808500003C80848001E14088800016B
:10055000540A880015220C84001443890700008186
:10056000060200000000000002FE01000002823FBF
:10057000FF00048202000004FE0200000C1004FCD4
:1005800000141004080005FF8C1000041014100063
:10059000043825FF00043404100004520410000441
:1005A0009184100005100450000410042000000085
:1005B0000000000000000000000000000002030036
:1005C00010001FDC3EFE000890021200051004FF20
:1005D000001FDF84120002120CFE001FD202100066
:1005E000021222FE000A921410000A521410001285
:1005F000220DFF0002220810000A4214100004021B
:1006000023FF00000000000000000000000F78BC85
:1006100020000948A45000094AA85000094AA888A7
:1006200000094AB104001FFEAAFB00094AA42000E9
:10063000094AA42000094AA7FE00094AB42000097B
:1006400048A924000B48A22200088AA4A20011197C
:10065000204000000000000000000000000020001A
:100660008000005001FC0000880104000104030820
:100670000006FB0490000800C0600007DF01800056
:10068000045106000004511BFE0004510202000741
:10069000D90202000456020200001003FE000010FE
:1006A000020200000000000000000000000208201C
:1006B0009000027F9890001F8009FF000222011025
:1006C0000006218B100007628DFE000AA2091000AF
:1006D0000A14111000121431FE0002081110000259
:1006E000141110000222111000024391FF00028138
:1006F00011000000000000000000000000100700D2
:10070000000008F83FFE0004802002000080200264
:100710000000BE23E2001C8222220004A422220048
:1007200004942222000488222200049423E200057B
:100730002220020005422002000A003FFE0011FFB5
:10074000A002000000000000000000000001041FE3
:10075000FC0000880080000FFF0080000020008067
:1007600000002000800000203FFF001FFF8080006D
:100770000020008000005000800000500080000039
:1007800088008000010400800006038280001801B8
:10079000010000000000000009FF00400004203FAD
:1007A000FF00042000000000FE0000001C420FFCBF
:1007B00000044200000007FF80000004000FFC005E
:1007C00004FF000000048100000005810FFC00060A
:1007D0008108040004FF08040000810FFC000000F1
:1007E00000000000000000000000000000004000C9
:1007F00080001FFF9FFC0000400410000FFF02203C
:100800000000003FFF000FFE00000008420FF8004C
:1008100008420808000FFE08080008020FF8000848
:1008200000080800080008080008000FF800100081
:100830000808000000000000000000000007FE0F94
:10084000F8000402000000040200000007FE00009F
:100850000004023FFE00040200800007FE0080004A
:10086000009004900008910C880006931086000206
:1008700094208200009000800000900280001FFF02
:1008800081000000000000000000000000041012C1
:10089000020005FF9FD20005009212001E28A2123E
:1008A0000004443FF200048202120006000212001B
:1008B0000CFE1FD200141012520004101242000449
:1008C00010134200041012820015FF820A00080073
:1008D00002040000000000000000000000002000F2
:1008E000000000203E04001FFFA204001000A2FF31
:1008F0000000012204000FFE22040000403E4400DC
:1009000000402224000440222400047C220400042D
:10091000402204000A403E0400094022240010FF47
:100920008014000000000800000000000010FE0815
:10093000200008820BFF0004820A010010FE3C51D7
:10094000000882088800088209040002FE0C0000EA
:10095000040019FC0009FF282000192908200009BB
:1009600029082000092908200009292BFF000BFF76
:10097000900000000000000000000000001F7F90B9
:10098000F80001080888000A10088800047F0107A1
:10099000001FC13A0000054909FC00044908840011
:1009A0000449088800044908480004490850000424
:1009B000490A200004160C5800142189870008C039
:1009C00086020000000000000FFFFFFFFFF03FFF66
:1009D000FFFFFFFC7FFFFFFFFFFE7FFFFFFFFFFE2C
:1009E000F0000000000FF0000000000FF000000019
:1009F000000FF1FFFFFFFF8FF1FFFFFFFF8FF1FF00
:100A0000FFFFFF8FF1FFFFFFFF8FF1FFFFFFFF8F62
:100A1000F1FFFFFFFF8FF1FFFFFFFF8FF1FFFFFFF0
:100A2000FF8FF1FFFFFFFF8FF1FFFFFFFF8FF1FF50
:100A3000FFFFFF8FF1FFFFFFFF8FF1FFFF03FF8F2E
:100A4000F1FFFF03FF8FF1FFFF03FF8FF1FFFFFFB8
:100A5000F18FF1FFFFFFE18FF1FFFFFFC78FF1FF84
:100A6000FFFF8F8FF1FFFFFF0F8FF1FFFFFF8F8FD2
:100A7000F1FFFFFFC78FF1FFFFFFE18FF1FFFFFFE6
:100A8000F18FF1FFFFFFFF8FF1FFFFFFFF8FF000FE
:100A90000000000FF0000000000FF0000000000F49
:100AA000F1FFFFFFFF8FF1111FFFFF8FF1111FFFFC
:100AB000FF8FF1111FFFFF8FF1FFFFFFFF8FF0008E
:100AC0000000000FF0000000000FF0000000000F19
:100AD0007FFFFFFFFFFE7FFFFFFFFFFE3FFFFFFFE8
:100AE000FFFC0FFFFFFFFFF00FFFFFFFFFF03FFFD7
:100AF000FFFFFFFC7FFFFFFFFFFE7FFFFFFFFFFE0B
:100B0000FFFFFFFFFFFFFFFFFFFFFFFFFFFFFFFFF5
:100B1000FFFFFFFFFFFFFFFFFFFFFFFFFFFFFFFFE5
:100B2000FFFFFFFFFFFFFFFFFFFFFFFFFFFFFFFFD5
:100B3000FFFFFFFFFFFFFFFFFFFFFFFFFFFFFFC7FD
:100B4000001FC00FFFC7001FC00C1FC7001FC00C35
:100B50001FC71FFFC7FC0FC71FFFC7FC4FC71FFFE3
:100B6000C7FC4FC71FFFC7FC47C71FFFC7FC67C7AE
:100B70001C01C01C63C71C01C01C73C71C01C01C26
:100B800071C71F8FC7FC79C71F8FC7FC78C71F8F1E
:100B9000C7FC7C071F8FC7FC7C07000FC00C7E07BB
:100BA000000FC00FFFFF000FC00FFFFFFFFFFFFF91
:100BB000FFFFFFFFFFFFFFFFFFFFFFFFFFFFFFFF45
:100BC000FFFFFFFFFFFFFFFFFFFFFFFFFFFFFFFF35
:100BD000FFFFFFFFFFFFFFFFFFFFFFFFFFFFFFFF25
:100BE000FFFFFFFFFFFFFFFFFFFFFFFFFFFFFFFF15
:100BF0007FFFFFFFFFFE7FFFFFFFFFFE3FFFFFFFC7
:100C0000FFFC0FFFFFFFFFF00FFFFFFFFFF03FFFB5
:100C1000FFFFFFFC7FFFFFFFFFFE7FFFFFFFFFFEE9
:100C2000FFFFFFFFFFFFFFFFFFFFFFFFFFFFFFFFD4
:100C3000FFFFFFFFFC7FFFFFFFFFFC7FFFFFFFFFCA
:100C4000FC7FFFFFFFFFFC7FFFFFFFFFFC7FFFFF3D
:100C5000FFFFFC7FFFFFFFFFFC7FFFFFFFFFFC7F2D
:100C6000FFFFFE00000001FFFE00000001FFFE008C
:100C7000000001FFFE3FFC7FF1FFFE3FFC7FF1FF24
:100C8000FE3FFC7FF1FFFE3FFC7FF1FFFE3FFC7F5C
:100C9000F1FFFE3FFC7FF1FFFE3FFC7FF1FFFE3FD7
:100CA000FC7FF1FFFE3FFC7FF1FFFE000000007FB4
:100CB000FE000000007FFE000000007FFE3FFC7F82
:100CC000FFFFFFFFFC7FFFFFFFFFFC7FFFFFFFFF3A
:100CD000FC7FFFFFFFFFFC7FFFFFFFFFFC7FFFFFAD
:100CE000FFFFFC7FFFFFFFFFFC7FFFFFFFFFFC7F9D
:100CF000FFFFFFFFFC7FFFFFFFFFFC7FFFFFFFFF0A
:100D0000FCFFFFFFFFFFFFFFFFFFFFFFFFFFFFFFF6
:100D10007FFFFFFFFFFE7FFFFFFFFFFE3FFFFFFFA5
:100D2000FFFC0FFFFFFFFFF00FFFFFFFFFF03FFF94
:100D3000FFFFFFFC7FFFFFFFFFFE7FFFC003FFFE03
:100D4000FFFF0000FFFFFFFC00003FFFFFF000007F
:100D50000FFFFFC0000003FFFFC0000001FFFF0006
:100D6000000000FFFF000000007FFE000000007F89
:100D7000FC000000003FFC000000203FF8000000E5
:100D8000701FF8000000F81FF0000001F80FF000DD
:100D90000003F00FF0000007E00FF000000FC00F9D
:100DA000E000001F8007E001803F0007E003C07EF5
:100DB0000007E007E0FC0007E003F1F80007E001AE
:100DC000FFF00007E000FFE00007E0007FC0000741
:100DD000F0003F80000FF0001F00000FF0000E0039
:100DE000000FF0000400000FF8000000001FF800E2
:100DF0000000001FFC000000003FFC000000003F5E
:100E0000FF000000007FFF00000000FFFF800000E7
:100E100001FFFFC0000003FFFFF0000007FFFFF02D
:100E200000000FFFFFFC00003FFFFFFF0000FFFF7F
:100E30007FFFF00FFFFE7FFFFFFFFFFE3FFFFFFF83
:100E4000FFFC0FFFFFFFFFF00FFFFFFFFFF03FFF73
:100E5000FFFFFFFC7FFFFFFFFFFE7FFFC001FFFEE4
:100E6000FFFF0000FFFFFFFC00001FFFFFF000007E
:100E70000FFFFFE0000003FFFFC0000001FFFF8045
:100E8000000000FFFF000000007FFE000000007F68
:100E9000FE000000003FFC008000801FF801C0033E
:100EA000C01FF803E003E01FF803F00FE00FF001AC
:100EB000F80FC007F000FC1F8007F0007E7F0007DE
:100EC000E0003FFE0007E0001FFC0007E0000FF815
:100ED0000007E00007F00007E00007F00007E0006F
:100EE0001FF80007E0001FFC0007E0007FFE00077E
:100EF000F0007E3F0007F001FC1F8007F001F80FB3
:100F0000C00FF803F007E00FF803E003E01FF8015B
:100F1000C001801FFE008000803FFE000000003FF7
:100F2000FF000000007FFF000000007FFF80000046
:100F300000FFFFC0000001FFFFF0000007FFFFF807
:100F400000000FFFFFFC00003FFFFFFF8000FFFFDE
:100F50007FFFF007FFFE7FFFFFFFFFFE3FFFFFFF6A
:100F6000FFFC0FFFFFFFFFF00FFFFFFFFFF03FFF52
:100F7000FFFFFFFC7FFFFFFFFFFE7FFFF00FFFFE85
:100F8000FFFFF00FFFFFFFFFE007FFBFFFFFC3C33F
:100F9000FF1FFFFF87E1FE0FFFFF0FF0FC1FFFFEAB
:100FA0001FF8783FFFFC3FFCF07FFFF87FFFE0FF7A
:100FB000FFF0FFFFC1FFFFE1FFFF83FFFFE3FFFF44
:100FC00007FFFFE3FFFE07FFFFE3FFFC07FFFFE371
:100FD000FFF807FFFFE3FFF047FFFFE3FFE0C7FF76
:100FE000FFE3FFC1C7FFFFE3FF83C7FFFFE3FF0787
:100FF000C7FFFFE3FE0FC7FFFFE3FC1FC7FFFFE3D1
:10100000F83FC7FFFFE3F07FC7FFFFE3E0FFC7FF45
:10101000FFE3C1FFC7FFFFE783FFC7FFFFEF07FF46
:10102000C7FFFFFE0FFFC1FFFFFC1FFFE0FFFFF840
:101030003FFFF87FFFF07FFFFC3FFFE00000003F35
:10104000FFC00000003FFF800000003FFF07FFFFE0
:10105000FFFFFE0FC003FFFFFC1FC003FFFFFE3FAB
:10106000E007FFFFFF7FE007FFFFFFFFF81FFFFF25
:101070007FFFF81FFFFE7FFFFFFFFFFE3FFFFFFF29
:10108000FFFC0FFFFFFFFFF00FFFFFFFFFF03FFF31
:10109000FFFFFFFC7FFFFFFFFFFE7FFFFFFFFFFE65
:1010A000F0000000000FF0000000000FF000000052
:1010B000000FF1FFFFFFFF8FF1FFFFF8888FF1FFB7
:1010C000FFF8888FF1FFFFF8888FF1FFFFFFFF8F98
:1010D000F0000000000FF0000000000FF000000022
:1010E000000FF1FFFFFFFF8FF10DDDFE4A8FF10AC8
:1010F000AAFFCD8FF10888FE5F8FF11AAAFFFF8F3C
:10110000F1FFFFFFFF8FF1FFFFFFFF8FF1FFFF00F8
:10111000008FF10C017FFF8FF16FFF46318FF16C73
:101120003F56B78FF11FFF56B78FF1FFFF46318F44
:10113000F1FFFF77B58FF1FFFF77B58FF10C0177E6
:10114000B58FF16FFF46318FF16C3F7FFF8FF11F3D
:10115000FF00008FF1FFFFFFFF8FF1FFFFFFFF8F09
:10116000F1FFFFFFFF8FF100002AA48FF10000556F
:10117000228FF1E0002AA48FF1FFFFFFFF8FF00024
:101180000000000FF0000000000FF0000000000F52
:101190007FFFFFFFFFFE7FFFFFFFFFFE3FFFFFFF21
:1011A000FFFC0FFFFFFFFFF00FFFFFFFFFF03FFF10
:1011B000FFFFFFFC7FFFFFFFFFFE7FFFFFFFFFFE44
:1011C000F0000000000FF0000000000FF000000031
:1011D000000FF1FFFFFFFF8FF1FFFFF8888FF1FF96
:1011E000FFF8888FF1FFFFF8888FF1FFFFFFFF8F77
:1011F000F0000000000FF0000000000FF000000001
:10120000000FF1FFFFFFFF8FF1FFFFFFFF8FF1FFE7
:10121000FFFFFF8FF1FFFFFFFF8FF1FFFFFFFF8F4A
:10122000F180F01F018FF180F01F018FF19CF39F7F
:10123000F98FF19CF39FF98FF19CF39FF98FF19C4B
:10124000F39FF98FF180F01C018FF180F01C018F6A
:10125000F1FCFF9CF98FF1FCFF9CF98FF1FCFF9CE6
:10126000F98FF1FCFF9CF98FF100E01C018FF10078
:10127000E01C018FF1FFFFFFFF8FF1FFFFFFFF8FEA
:10128000F1FFFFFFFF8FF1FFFFFFFF8FF1FFFFFF78
:10129000FF8FF1FFFFFFFF8FF1FFFFFFFF8FF000D8
:1012A0000000000FF0000000000FF0000000000F31
:1012B0007FFFFFFFFFFE7FFFFFFFFFFE3FFFFFFF00
:1012C000FFFC0FFFFFFFFFF00FFFFFFFFFF03FFFEF
:1012D000FFFFFFFC7FFFFFFFFFFE7FFFFFFFFFFE23
:1012E000FFFFFFFFFFFFFDFFFFFFFFFFF8FFFFFF17
:1012F000FFFFF07FFFFFFFFFE03FFFFFFFFFF8FF73
:10130000FFFFFFFFF8FFFFFFFFFFF8FFFFFFFFFFFB
:10131000F8E7FFFFFFFFF8E7FFE1FFFFF8E3FF005B
:101320007FFFF8F3FE0C1FFFF8F3F87F0FFFF8F1D3
:10133000F0FFC7FFF8F9E3FFE3FFF8F8E7FFF1FF7D
:10134000F8FC47FFF8FFF8FE0FFFFCFFF8FF1FFF58
:10135000FFFFF8FF1FFFFFFFF8FE0FFFFFFFF8FE84
:1013600047FFFFFFF8FC63FFFFFFF8FCF0FFFFFF04
:10137000F8F8F87FFFFFF8F9FE1FFFFFF8F1FF070D
:10138000FFFFF8E3FFC1FFFFF8C7FFF01FFFF8C73B
:10139000FFFC07FFF8CFFFFFC7FFF8FFFFFFFFFFCE
:1013A000F8FFFFFFFFFFF8FFFFFFFFBFF8FFFFFFA2
:1013B000FF9FF8000000000FF80000000007F80091
:1013C0000000000FFFFFFFFFFF9FFFFFFFFFFFBFBA
:1013D0007FFFFFFFFFFE7FFFFFFFFFFE3FFFFFFFDF
:1013E000FFFC0FFFFFFFFFF00FFFFFFFFFF03FFFCE
:1013F000FFFFFFFC7FFFFFFFFFFE7FFFFFFFFFFE02
:10140000FFFFFFFFFFFFFDFFFFFFFFFFF8FFFFFFF5
:10141000FFFFF07FFFFFFFFFE03FFFFFFFFFF8FF51
:10142000FFFFFFFFF8FFFFFFFFFFF8FFFFFFFFFFDA
:10143000F8E7FFFFFFFFF8E7C00003FFF8E3C00095
:1014400003FFF8F3CFFFFFFFF8F3CFFFFFFFF8F143
:10145000CFFFFFFFF8F9CFFFFFFFF8F8CFFFFFFF47
:10146000F8FC4FFFFFFFF8FE0FFFFFFFF8FF0FFF35
:10147000FFFFF8FF0FFFFFFFF8FF8FFFFFFFF8FFF1
:10148000C7FFFFFFF8FFC3FFFFFFF8FFC0FFFFFF2D
:10149000F8FFC87FFFFFF8800E1FFFFFF8800F07DF
:1014A000FFFFF8FFFFC1FFFFF8FFFFF01FFFF8FF8E
:1014B000FFFC07FFF8FFFFFFC7FFF8FFFFFFFFFF7D
:1014C000F8FFFFFFFFFFF8FFFFFFFFBFF8FFFFFF81
:1014D000FF9FF8000000000FF80000000007F80070
:1014E0000000000FFFFFFFFFFF9FFFFFFFFFFFBF99
:1014F0007FFFFFFFFFFE7FFFFFFFFFFE3FFFFFFFBE
:10150000FFFC0FFFFFFFFFF00FFFFFFFFFF03FFFAC
:10151000FFFFFFFC7FFFFFFFFFFE7FFFFE3FFFFEA1
:10152000FFFFFE3FFFFFFFFFFE3FFFFFFFFFFE3F0E
:10153000FFFFFFFFFE3FFFFFFFFFBE3DFFFFFFFE80
:101540003E3C7FFFFFFC3E3C3FFFFFF83E3C1FFF61
:10155000FFF0FE3F0FFFFFE1FE3F87FFFFC3FE3FAF
:10156000C3FFFF87FE3FE1FFFF8FFE3FF1FFFF0F4D
:10157000FE3FF0FFFF1FFE3FF8FFFF1FFE3FF8FF9B
:10158000FE1FFE3FFC7FFE3FFE3FFC7FFE3FFE3F17
:10159000FC7FFE3FFE3FFC7FFE3FFE3FFC7FFE3FA9
:1015A000FFFFFC7FFE3FFFFFFC7FFE1FFFFFFC7F76
:1015B000FF1FFFFFF8FFFF1FFFFFF8FFFF0FFFFFF9
:1015C000F0FFFF8FFFFFF1FFFF87FFFFE1FFFFC38A
:1015D000FFFFC3FFFFE1FFFF87FFFFF0FFFF07FFF4
:1015E000FFF83FFC0FFFFFFC0FF03FFFFFFE000086
:1015F0007FFFFFFF8001FFFFFFFFF00FFFFFFFFFF7
:10160000FFFFFFFFFFFFFFFFFFFFFFFFFFFFFFFFEA
:101610007FFFFFFFFFFE7FFFFFFFFFFE3FFFFFFF9C
:10162000FFFC0FFFFFFFFFF00FFFFFFFFFF03FFF8B
:10163000FFFFFFFC7FFEFFFFFFFE7FFE7FFFFFFE41
:10164000FFFE3FFFFFFFFFFE1FFFFFFFFFFE0FFF3D
:10165000FFFFFFFE07FFFFFFFFFE03FFFFFFFFFE91
:1016600001FFFFFFFFFE01FFFFFFFFFC00FFFFFF89
:10167000FFF800FFFFFFFFF000FFFFFFFFE0007F2C
:10168000FFFFFFE0007FFFFFFFC0007FFFFFFF8045
:10169000007FFFFFFF00007EFFFFFF00007E7FFF57
:1016A000FE0000FE3FFFFC0000FF1FFFFC0000FEED
:1016B0000FFFF80001FE07FFF80001FE03FFF00036
:1016C00003FC01FFF00007FC01FFF0000FF801FF31
:1016D000F0001FF000FFF0001FF000FFF0003FE0FF
:1016E000007FF8007FC0007FF800FF80007FFC00D3
:1016F000FF00007FFC01FF00007FFE01FE00007F75
:10170000FE03FC00007FFF03F80000FFFF83F800EA
:1017100000FFFFC7F80000FFFFE3F00001FFFFF349
:10172000F00003FFFFFFF00007FFFFFFFFFFFFFFD9
:101730007FFFFFFFFFFE7FFFFFFFFFFE3FFFFFFF7B
:10174000FFFC0FFFFFFFFFF00FFFFFFFFFF03FFF6A
:10175000FFFFFFFC7FFFFFFFFFFE7FFFFFC1FFFEDC
:10176000FFFFFF01FFFFFFFFFC01FFFFFFFFF00195
:10177000FFFFFFFFC001FFFFFFFF0007FFFFFFFCB0
:10178000001FFFFFFFF0007F9FFFFFE001FE0FFF44
:10179000FFC007F807FFFFC01FE007FFFFC07F8003
:1017A00007FFFFE1FE001FFFFFFFF8003FFFFFFF05
:1017B000E001FFFFFFFF8003FFFFFFFE000FFFFFC1
:1017C000FFF8003FFFFFFFE000FE0FFFFFC003FC3C
:1017D00007FFFFC00FE007FFFFC03FC007FFFFC0CC
:1017E000FE000FFFFFFFFC003FFFFFFFE0007FFF59
:1017F000FFFFC003FFFFFFFF0001FFFFFFFE00012F
:10180000FFFFFFFE0000FFFFFFFE0001FFFFFFFFE5
:101810000001FFFFFFFFFFFFFFFFFFFFFFFFFFFFD5
:10182000FFFFFFFFFFFFFFFFFFFFFFFFFFFFFFFFC8
:10183000FFFFFFFFE00FFFFFFFFFC007FFFFFFFFFE
:101840008007FFFFFFFF8007FFFFFFFFC00FFFFFC5
:101850007FFFE01FFFFE7FFFFFFFFFFE3FFFFFFF59
:10186000FFFC0FFFFFFFFFF00FFFFFFFFFF03FFF49
:10187000FFFFFFFC7FFFFFFFFFFE7FFFFFFFFFFE7D
:10188000F00000001FFFF00000000FFFF00000005C
:1018900007FFF1C00FF8C3FFF1C00FF8E1FFF1C07F
:1018A0000FF8F0FFF1C00FF8F87FF1C00FF8FC3F20
:1018B000F1C00FF8FE1FF1C00000FF0FF1C00000E3
:1018C000FF8FF1C00000FF8FF1FFFFFFFF8FF1FFDF
:1018D000FFFFFF8FF1FFFFFFFF8FF1FFFFFFFF8F84
:1018E000F1FFFFFFFF8FF1FFFFFFFF8FF1FFFFFF12
:1018F000FF8FF1FFFFFFFF8FF1FFFFFFFF8FF1C0B1
:101900000000038FF1C00000038FF1C00000038FBF
:10191000F1C7FFFFE38FF1C7FFFFE38FF1C60000C0
:10192000E38FF1C60000E38FF1C60000E38FF1C73B
:10193000FFFFE38FF1C7FFFFE38FF1C60000E38FE6
:10194000F1C60000E38FF1C60000E38FF1C7FFFF8F
:10195000E38FF1C7FFFFE38FF1C7FFFFE38FF000D5
:101960000000000FF0000000000FF0000000000F6A
:101970007FFFFFFFFFFE7FFFFFFFFFFE3FFFFFFF39
:10198000FFFC0FFFFFFFFFF00FFFFFFFFFF03FFF28
:10199000FFFFFFFC7FFFFFFFFFFE7FFFFFFFFFFE5C
:1019A000FFFFFFFFFFFFFFFFFFFFFFFFFFFFFFFF47
:1019B000FFFFFFFFFFFFFFFFFFFFFFFFFFFFFFFF37
:1019C000FFFFFFFFFFFFFFFFFFFFFFFFFE3FFFFFE8
:1019D000FFFFFE3FFFFFFFFFFE3FFFFFFFFFFE3F5A
:1019E000FFFFFFFFFE3FFFFFFFFFFE3FFFFFFFFF89
:1019F000FE3FFFFFFFFFFE3FFFFFFFFFFE3FFFFF3A
:101A0000FFFFFE3FFFFFFFFFFE3FFFFFFFF0000075
:101A10000FFFFFF000000FFFFFF000000FFFFFFFC0
:101A2000FFFFFFFFFFFFFE3FFFFFFFFFFE3FFFFF48
:101A3000FFFFFE3FFFFFFFFFFE3FFFFFFFFFFE3FF9
:101A4000FFFFFFFFFE3FFFFFFFFFFE3FFFFFFFFF28
:101A5000FE3FFFFFFFFFFE3FFFFFFFFFFFFFFFFF18
:101A6000FFFFFFFFFFFFFFFFFFFFFFFFFFFFFFFF86
:101A7000FFFFFFFFFFFFFFFFFFFFFFFFFFFFFFFF76
:101A8000FFFFFFFFFFFFFFFFFFFFFFFFFFFFFFFF66
:101A90007FFFFFFFFFFE7FFFFFFFFFFE3FFFFFFF18
:101AA000FFFC0FFFFFFFFFF00FFFFFFFFFF03FFE08
:101AB00000007FFC7FFE00007FFE7FFC00003FFEF9
:101AC000FFFC7FFE3FFFFFFC7FFE3FFFFFFC7FFE32
:101AD0003FFFFC000000001FF8000000000FF000B6
:101AE00000000007F1FFFFFFFFC7F1FFFFFFFFC787
:101AF000F1FFFFFFFFC7F00000000007F800000043
:101B0000000FFC000000001FFFFFFFFFFFFFFC7F36
:101B1000FFFFFE3FFC7FFFFFFE3FFC7FFFFFFE3F1E
:101B2000FC7F8FF8FE3FFC7F8FF8FE3FFC7F8FF835
:101B3000FE3FFC7F8FF8FE3FFC7F8FF8FE3FFC7F6F
:101B40008FF8FE3FFC7F8FF8FE3FFC7F8FF8FE3F53
:101B5000FC7F8FF8FE3FFC7F8FF8FE3FFC7F8FF805
:101B6000FE3FFC7F8FF8FE3FFC7F8FF8FE3FFC7F3F
:101B70008FF8FE3FFC7F8FF8FE3FFC7F8FF8FE3F23
:101B8000FC7F8FF8FE3FFC7FFFFFFE3FFC7FFFFFE7
:101B9000FE3FFC7FFFFFFE3FFC7FFFFFFE3FFC7F21
:101BA000FFFFFE3FFC3FFFFFFC3FFC000000003F4B
:101BB0007E000000007E7F00000000FE3FFFFFFF70
:101BC000FFFC0FFFFFFFFFF00FFFFFFFFFF03FFFE6
:101BD000FFFFFFFC7FFFFFFFFFFE7FFFFFFFFFFE1A
:101BE000FFFFFFFFFFFFFFFFFFFFFFFFFFFFFFFF05
:101BF000FFFFFFFFF007FFFFFFFF8000FFFFFFFE7B
:101C000000003FFFFFF807F00FFFFFF03FFE07FF68
:101C1000FFE0FFFF83FFFFC1FFFFE1FFFF87FFFF43
:101C2000F0FFFF0FFFFFF87FFF0FFFFFFC7FFE1F9E
:101C3000FFFFFC3FFE3FFFFFFE3FFC3FF3FBFE1FAD
:101C4000FC7FE1F0FF1FFC7FC0E07F1FF87F80403A
:101C50007F0FF8FF00003F8FF8FF00003F8FF8FF75
:101C600000001F8FF8FE00001F8FFFFE00001FFF07
:101C7000FFFE00001FFFFFFE00001FFFFFFF000030
:101C80001FFFFFFF00003FFFFFFF00003FFFFFFFC0
:101C900080007FFFFFFF80007FFFFFFFC000FFFF8E
:101CA000FFFFF003FFFFFFFFFC0FFFFFFFFFFFFF42
:101CB000FFFFFFFFFFFFFFFFFFFFFFFFFFFFFFFF34
:101CC000FFFFFFFFFFFFFFFFFFFFFFFFFFFFFFFF24
:101CD0007FFFFFFFFFFE7FFFFFFFFFFE3FFFFFFFD6
:101CE000FFFC0FFFFFFFFFF00FFFFFFFFFF03FFFC5
:101CF000FFFFFFFC7FFFFFFFFFFE600000001FFEF5
:101D0000E00000001FFFE00000001FFFE3FFFFFFF7
:101D10001FFFE3FFFFFF1FFFE3FFFFFF10FFE3FFD6
:101D2000FFFF10FFE3FFFFFF10FFE3FFFFFF18FFC0
:101D3000E3FFFFFF18FFE3FFFFFF1887E3FFFFFF4D
:101D40001887E3FFFFFF1887E3FFFFFF18C7E3FFD4
:101D5000FFFF18C7E3FFFFFF18C7E3FFFFFF18C728
:101D6000E3FFFFFF18C7E3FFFFFF18C7E3FFFFFF15
:101D700018C7E3FFFFFF18C7E3FFFFFF18C7E3FF24
:101D8000FFFF18C7E3FFFFFF18C7E3FFFFFF18C7F8
:101D9000E3FFFFFF18C7E3FFFFFF18C7E3FFFFFFE5
:101DA00018C7E3FFFFFF18C7E000000018C7E000F6
:101DB000000018C7E000000018C7FFFFFFFFF8C7CA
:101DC000FF1FFFFFF8C7FF00000000C7FF00000073
:101DD00000C7FF00000000C7FFFFFFFFFFC7FFF8BD
:101DE000FFFFFFC7FFF800000007FFF80000000733
:101DF0007FF8000000067FFFFFFFFFFE3FFFFFFFB1
:101E0000FFFC0FFFFFFFFFF00FFFFFFFFFF03FFFA3
:101E1000FFFFFFFC7FFFFFFFFFFE7FFFFFFFFFFED7
:101E2000FFFFFFFFFFFFF000007FFFFFF000007FDC
:101E3000FFFFF000007FFFFFF1FFFFFFFF0FF1FF4B
:101E4000FFFFFE0FF1FFFFFFFC0FF1FFFFFFF81F89
:101E5000F1FFFFFFF03FF1FFFFFFE07FF1FFFFFF2A
:101E6000C0FFF1FFFFFF81FFF1FFFFFF03FFF1FF65
:101E7000FFFE07FFF1FFFFFC0FFFF1FE1FF81FFF42
:101E8000F1FE0FF03FFFF1FE07E07FFFF1FE03C020
:101E9000FFFFF1FF0181FFFFF1FF8003FFFFF1FF73
:101EA000C007FC7FF1FFE00FFC7FF1FFF01FFC7F1C
:101EB000F1FFF83FFC7FF1FFFC7FFC7FF1FFFFFFAC
:101EC000FC7FF1FFFFFFFC7FF1FFFFFFFC7FF1FFD5
:101ED000FFFFFC7FF1FFFFFFFC7FF1FFFFFFFC7FB7
:101EE000F1FFFFFFFC7FF1FFFFFFFC7FF1FFFFFF32
:101EF000FC7FF0000000007FF0000000007FF00099
:101F00000000007FFFFFFFFFFFFFFFFFFFFFFFFF5E
:101F10007FFFFFFFFFFE7FFFFFFFFFFE3FFFFFFF93
:101F2000FFFC0FFFFFFFFFF00FFFFFFFFFF03FFF82
:101F3000FFFFFFFC7FFFFFFFFFFE7FFFFFFFFFFEB6
:101F4000FFFFFFFFFFFFFFFFFF1FFFFFFFFFFE0F72
:101F5000FFFFFFFFFE0FFFFFFFFFFE0FFFFFFFFF73
:101F6000FF1FFFFFFFFFFFFFFFFFFFFFFFFFFFFF61
:101F7000FFFFFFFFFFFFFFFFFFFFFFFFFFFFFFFF71
:101F8000FFFFFFFFC00FFFFFFFFF8007FFFFFFFF07
:101F90000007FFFFFFFE0F87FFFFFFFE1FC7FFFFCA
:101FA000FFFE3FC7FFFFFFFE3FC7FFFFFFFFFFC76B
:101FB000FFFFFFFFFFC7FFFFFFFFFFC7FFFFFFFFA1
:101FC000FF87FFFFFFFFFF0FFFFFFFFFFE1FFFFF6A
:101FD000FFFFFC3FFFFFFFFFF87FFFFFFFFFF0FF6A
:101FE000FFFFFFFFF1FFFFFFFFFFF1FFFFFFFFFF1D
:101FF000F1FFFFFFFFFFF1FFFFFFFFFFF1FFFFFF1B
:10200000FFFFF1FE3FFFFFFFF0FE3FFFFFFFF87C09
:102010003FFFFFFFFC003FFFFFFFFE007FFFFFFFD2
:10202000FF00FFFFFFFFFFFFFFFFFFFFFFFFFFFFBF
:102030007FFFFFFFFFFE7FFFFFFFFFFE3FFFFFFF72
:10204000FFFC0FFFFFFFFFF00FFFFFFFFFF03FFF61
:10205000FFFFFFFC7FFFC001FFFE7FFE00007FFE51
:10206000FFF800001FFFFFE0000007FFFFC0400275
:1020700003FFFF81800181FFFF078420E0FFFE0F47
:102080000C30F07FFC1E0C38783FF83E1C387C1F6B
:10209000F87C1C3C3E1FF07C3C3C3F0FF0FC3C3E7F
:1020A0001F0FE1F87C3E1F87E1F87C3E1F87E1F8B7
:1020B0007C3F1FC7C3F8FC3F0FC3C3F0FC3F0FC3F7
:1020C000C3F0FC3F0FC3C00000000003C0000000CD
:1020D0000003C00000000003C00000000003C7F0C0
:1020E000FC3F0FE3C3F0FC3F0FE3C3F0FC3F0FC323
:1020F000C3F0FC3F0FC3C3F0FC3F0FC3E1F8FC3F4C
:102100001FC7E1F87C3E1F87E1F87C3E1F87F0FC8B
:102110007C3E3F0FF07C3C3C3E0FF87C3C3C3E1F3D
:10212000FC3E1C387C3FFC1E0C30783FFE0F0C3010
:10213000F07FFF030420C0FFFF81800181FFFFC00B
:10214000000003FFFFF000000FFFFFF800001FFF7B
:102150007FFE00007FFE7FFFC003FFFE3FFFFFFF0B
:10216000FFFC0FFFFFFFFFF00FFFFFFFFFF03FFF40
:10217000FFFFFFFC7FFFFFFFFFFE7FFFF00FFFFE73
:10218000FFFFF00FFFFFFFFFE007FFFFFFFFC3C3ED
:10219000FFFFFFFF87E1FFFFFFFF0FF0FFFFFFFEE5
:1021A0001FF87FFFFFFC3FFC3FFFFFF87FFE1FFF94
:1021B000FFF0FFFF0FFFFFE1FFFF87FFFFE3FFFFE0
:1021C000C7FFFFE3FFFFC7FFFFE3FFFFC7FFFFE31B
:1021D000FFFFC7FFFFE3FFFFC7FFFFE3FFFFC7FFEF
:1021E000FFE3FFFFC7FFFFE3FFFFC7FFFFE3FFFFC3
:1021F000C7FFFFE3FFFFC7FFFFE3FFFFC7FFFFE3EB
:10220000FFFFC7FFFFE3FFFFC7FFFFE3FFFFC7FFBE
:10221000FFE3FFFFC7FFFFE3FFFFC7FFFFE3FFFF92
:10222000C7FFFF83FFFFC1FFFF07FFFFE0FFFE1FA8
:10223000FFFFF87FFC3FFFFFFC3FFC000000003F7A
:10224000FC000000003FFC000000003FFFFFFFFF1C
:10225000FFFFFFFFC003FFFFFFFFC003FFFFFFFF04
:10226000E007FFFFFFFFE007FFFFFFFFF81FFFFF93
:102270007FFFF81FFFFE7FFFFFFFFFFE3FFFFFFF17
:10228000FFFC0FFFFFFFFFF00FFFFFFFFFF03FFF1F
:10229000FFFFFFFC7FFFFFFFFFFE7FFFFFFFFFFE53
:1022A000F0000000000FF0000000000FF000000040
:1022B000000FF1FFFFFFFF8FF1FFFFF8888FF1FFA5
:1022C000FFF8888FF1FFFFF8888FF1FFFFFFFF8F86
:1022D000F0000000000FF0000000000FF000000010
:1022E000000FF1FFFFFFFF8FF1FFFFFFFF8FF18F67
:1022F000FFFFFF8FF187FFFFFF8FF1E3FFFFFF8FEE
:10230000F1F1FFFFFF8FF1F0FFFFFF8FF1F1FFFF12
:10231000FF8FF1E3FFFFFF8FF187FFFFFF8FF18F4B
:10232000FFFFFF8FF1FFC0FFFF8FF1FFC0FFFF8FA7
:10233000F1FFC0FFFF8FF1FFFFFFFF8FF1FFFFFFF6
:10234000FF8FF1FFFFFFFF8FF1FFFFFFFF8FF1FF17
:10235000FFFFFF8FF1FFFFFFFF8FF1FFFFFFFF8FF9
:10236000F1FFFFFFFF8FF1FFFFFFFF8FF1FFFFFF87
:10237000FF8FF1FFFFFFFF8FF1FFFFFFFF8FF000E7
:102380000000000FF0000000000FF0000000000F40
:102390007FFFFFFFFFFE7FFFFFFFFFFE3FFFFFFF0F
:1023A000FFFC0FFFFFFFFFF00FFFFFFFFFF03FFFFE
:1023B000FFFFFFFC7FFFFF803FFE7FFFFF003FFE30
:1023C000FFFFFE007FFFFFFFFC00FFFFFFFFF801A4
:1023D000FFFFFFFFF003FFFFFFFFE007FFFFFFFF2F
:1023E000C007FFFFFFFFC007FFFFFFFFC007FFFFA2
:1023F000FFFFC007FFFFFFFFC007FFFFFFFFC00792
:10240000FFE7FFFFC007FFC7FFFFC007FF87FFFF12
:10241000C007FF07FFFFC007FE07FFFFC000000760
:10242000FFFFC0000007FFFFC000000FFFFF80009C
:10243000000FFFFF0000001FFFFE0000003FFFFC39
:102440000000007FFFF8000000FFFFF0000001FF28
:10245000FFE0000003FFFFC0000007FFFF80007FD8
:10246000FFFFFF0000FFFFFFFE0001FFFFFFFC007A
:1024700003FFFFFFF80007FFFFFFF0000FFFFFFF64
:10248000E0001FFFFFFFC3803FFFFFFF87C07FFF0C
:10249000FFFF87C0FFFFFFFF87C1FFFFFFFF8383B1
:1024A000FFFFFFFFC007FFFFFFFFC00FFFFFFFFFA2
:1024B000601FFFFFFFFE783FFFFFFFFE3FFFFFFFB4
:1024C000FFFC0FFFFFFFFFF00FFFFFFFFFF03FFFDD
:1024D000FFFFFFFC7FFFFFFFFFFE7FC7FFFFF1FE57
:1024E000FF03FFFFE07FFE03FFFFE03FFC03FFFF72
:1024F000E01FF807F007F00FF00F8000F807E01E6C
:1025000000003C03E03C00001E03E07000000703F5
:10251000E0E000000383F1C001C001C7FF8003E0D9
:1025200000FFFF8003E000FFFF0003E0007FFF00EB
:1025300003E0007FFE0003E0003FFE0003E0003FF9
:10254000FC0003E0001FFC0003E0001FFC0003E0B0
:10255000001FFC0003E0001FFC0003E0001FFC0064
:1025600003F0001FFC0001F8001FFC0000FC001F2E
:10257000FC00003E001FFE00001F003FFE00000F99
:10258000803FFF000007803FFF000003007FFF80C7
:10259000000000FFFF80000000FFFF80000000FF40
:1025A000FF000000007FFE000000003FFC00000074
:1025B000001FFC060000301FFC0F8000F81FFE1FEC
:1025C000F007FC3FFFFFFFFFFFFFFFFFFFFFFFFFE5
:1025D0007FFFFFFFFFFE7FFFFFFFFFFE3FFFFFFFCD
:1025E000FFFC0FFFFFFFFFF00FFFFFFFFFF03FFFBC
:1025F000FFFFFFFC7FFFF83FFFFE7FFFF01FFFFEA6
:10260000FFFFE38FFFFFFFFFE7CFFFFFFFFFE7CFF6
:10261000FFFFFFFFE7CFFFFFFFFFE1CFFFFFFFFF60
:10262000E1CFFFFFFFFFE7CFFFFFFFFFE7CFFFFF98
:10263000FFFFE7CFFFFFFFFFE7CFFFFFFFFFE1CF88
:10264000FFFFFFFFE1CFFFFFFFFFE7CFFFFFFFFF30
:10265000E7CFFFFFFFFFE7CFFFFFFFFFE7CFFFFF62
:10266000FFFFE1CFFFFFFFFFE1CFFFFFFFFFE7CF5E
:10267000FFFFFFFFE7CFFFFFFFFFE3CFFFFFFFFFFE
:10268000E0CFFFFFFFFFE00FFFFFFFFFE00FFFFFC7
:10269000FFFFE00FFFFFFFFFE00FFFFFFFFFE00F77
:1026A000FFFFFFFFE00FFFFFFFFFE00FFFFFFFFF58
:1026B000E00FFFFFFFFFC007FFFFFFFF8003FFFFEB
:1026C000FFFF8003FFFFFFFF8003FFFFFFFF80038B
:1026D000FFFFFFFF8003FFFFFFFF8003FFFFFFFF00
:1026E000C007FFFFFFFFC007FFFFFFFFE00FFFFF77
:1026F0007FFFF01FFFFE7FFFFFFFFFFE3FFFFFFF9B
:10270000FFFC0FFFFFFFFFF00FFFFFFFFFF03FFF9A
:10271000FFFFFFFC7FFFFFFFFFFE70003FFFFFFE9C
:10272000F0001FFFFFFFF0000FFFFFFFF00007FFAB
:10273000FFFFF00003FFFFFFF00001FFFFFFF00FBE
:1027400080FFFFFFF01FC07FFFFFF03FE03FFFFF74
:10275000F07FF01FFFFFF07FF00FFFFFF07FF0072B
:10276000FFFFF07FF003FFFFF03FE001FFFFF03FCE
:10277000E000FFFFF01FC0007FFFF00F80003FFF71
:10278000F80000001FFFFC0000000FFFFE0000002B
:1027900007FFFF00000003FFFF80000001FFFFC0F4
:1027A000000000FFFFE00000007FFFF00000003F9E
:1027B000FFF80000001FFFFC0000000FFFFE0000FC
:1027C0000007FFFF00000003FFFF80000007FFFF7E
:1027D000C000000FFFFFE000001FFFFFF000003F00
:1027E000FFFFF800007FFFFFFC0000FFFFFFFE007F
:1027F00001FFFFFFFF0003FFFFFFFF8007FFFFFF59
:10280000FFC00FFFFFFFFFE01FFFFFFFFFF03FFFD5
:102810007FFFFFF87FFE7FFFFFFCFFFE3FFFFFFF14
:10282000FFFC0FFFFFFFFFF0000007E01FF8181884
:102830001818181800003FFC3C3C3C3C3C3C3E7CDB
:102840003E7C3FFC3FFC00000400060007000F0038
:102850000F801F803F907F187F1C7E3C7C3E787EDF
:1028600078FE31FE11FC09F80FE01FF83FFC7FFEF7
:10287000FFE6FFCEFF9FF33FF07FF8FFFDFE7FFEF8
:102880007FFC3FF81FF003C000E003C00F001C38BE
:1028900010F003C00F001C3810F003E007E007E061
:1028A0000000000003C003800180018001801990B6
:1028B00039B8318C618C618660066006600E700CE0
:1028C000301C1C780FF003C00380038003C007C0D6
:1028D00007E00FE00E701E701E701E783FF83FFC80
:1028E0007E7C7E7E7FFE7FFE1140820021208FE075
:1028F00023FC82004A23E200FE209FF013F8808030
:102900002220C0804221BFF0FBFA88800220848010
:10291000022084801A208080E3FE82800201010070
:102920000F421FC0784110400840904008421FC02D
:1029300008411040FFFD104008405FC00840800083
:1029400008413FE008432520104125201041252063
:102950002041252040417FF07FF848800200490057
:102960000201FFF00201001002027F20220041005C
:1029700023F07F00220008002200FF8022008880D0
:102980002200888022008A8022008900FFFC080043
:1029900023F21FC022111040FBF0904022121FC0F2
:1029A0002A11104033F1104060005FC0AFFC80007E
:1029B00020413FE022432520227925202241252065
:1029C000A541252048FD7FF01083DFC010825040D4
:1029D000208250402FFFDFC06082520061C252004F
:1029E000A1C25FE022A3D20022A251002492510092
:1029F000288E5090308BD450208258302080101078
:102A0000104047C017FC44402003F44023F84440E2
:102A10006208C440A3F8E440200154402FFD444024
:102A20002806444023F84440204044502040485069
:102A3000214050302080400020921FC03DF990403E
:102A40002090904040901FC07BFF0000A0013FE01D
:102A500021F90200FD09020021097FF021F905009A
:102A6000210945002909888031F9107021082020AA
:102A700025004300202070F83F3F3F0053617665FA
:102A800000466C6970004D61696E20536372656524
:102A90006E004F4B004E4F00454E00434E005945CF
:102AA00053004E4F004F4E004F464600496E666F32
:102AB0007300426967005049440044697265637459
:102AC000005361766500426F6F7374004F66660055
:102AD000536C656570005361766500426F6F737467
:102AE00000536C6565700044656661756C740053D5
:102AF000617665004164640044656C6574650052EC
:102B0000656E616D650043616C6962726174650038
:102B10004368616E67650052657475726E0041624C
:102B20006F7574004C616E670042757A7A65720049
:102B300053637265656E00436F6E74726F6C005400
:102B4000696D65720054656D7000546970003E00D7
:102B500053656C65637420546970000000000000C8
:102B60003E5B4F5B3E3E6B4F6B3E1C3E7C3E1C18FB
:102B70003C7E3C181C577D571C1C5E7F5E1C001859
:102B80003C1800FFE7C3E7FF0018241800FFE7DB4D
:102B9000E7FF30483A060E2629792926407F0505A9
:102BA00007407F05253F5A3CE73C5A7F3E1C1C08E6
:102BB000081C1C3E7F14227F22145F5F005F5F06AB
:102BC000097F017F006689956A606060606094A2F9
:102BD000FFA29408047E040810207E201008082A12
:102BE0001C08081C2A08081E101010100C1E0C1EB1
:102BF0000C30383E3830060E3E0E06000000000055
:102C000000005F00000007000700147F147F1424F9
:102C10002A7F2A122313086462364956205000087E
:102C2000070300001C2241000041221C002A1C7FD7
:102C30001C2A08083E0808008070300008080808B0
:102C400008000060600020100804023E5149453E23
:102C500000427F400072494949462141494D33189D
:102C600014127F1027454545393C4A4949314121D5
:102C70001109073649494936464949291E000014B9
:102C80000000004034000000081422411414141401
:102C900014004122140802015909063E415D594EB3
:102CA0007C1211127C7F494949363E414141227FC5
:102CB0004141413E7F494949417F090909013E415E
:102CC0004151737F0808087F00417F410020404147
:102CD0003F017F081422417F404040407F021C0298
:102CE0007F7F0408107F3E4141413E7F090909066C
:102CF0003E4151215E7F091929462649494932033F
:102D0000017F01033F4040403F1F2040201F3F40C4
:102D100038403F631408146303047804036159497D
:102D20004D43007F414141020408102000414141D0
:102D30007F040201020440404040400003070800B5
:102D400020545478407F2844443838444444283838
:102D50004444287F385454541800087E090218A4AB
:102D6000A49C787F0804047800447D400020404003
:102D70003D007F1028440000417F40007C0478041F
:102D8000787C080404783844444438FC1824241817
:102D900018242418FC7C08040408485454542404BF
:102DA000043F44243C4040207C1C2040201C3C40EC
:102DB00030403C44281028444C9090907C4464540B
:102DC0004C440008364100000077000000413608FE
:102DD0000002010204023C2623263C1EA1A161122E
:102DE0003A4040207A38545455592155557941215B
:102DF00054547841215554784020545579400C1E44
:102E000052721239555555593954545459395554EB
:102E100054580000457C410002457D420001457C3C
:102E200040F0292429F0F0282528F07C545545004D
:102E30002054547C547C0A097F4932494949323232
:102E400048484832324A4848303A4141217A3A4269
:102E5000402078009DA0A07D39444444393D404045
:102E6000403D3C24FF2424487E4943662B2FFC2F01
:102E70002BFF0929F620C0887E090320545479418C
:102E80000000447D413048484A32384040227A00B0
:102E90007A0A0A727D0D19317D2629292F282629C3
:102EA00029292630484D4020380808080808080815
:102EB00008382F10C8ACBA2F102834FA00007B0055
:102EC0000008142A142222142A14089500220095BE
:102ED000AA005500AAAA55AA55AA000000FF001092
:102EE0001010FF00141414FF001010FF00FF10104A
:102EF000F010F0141414FC001414F700FF0000FF8D
:102F000000FF1414F404FC141417101F10101F10E9
:102F10001F1414141F00101010F0000000001F10E8
:102F20001010101F10101010F010000000FF1010F3
:102F300010101010101010FF10000000FF140000FF
:102F4000FF00FF00001F10170000FC04F41414170A
:102F500010171414F404F40000FF00F714141414F0
:102F6000141414F700F7141414171410101F101F62
:102F7000141414F4141010F010F000001F101F00AF
:102F800000001F14000000FC140000F010F01010EE
:102F9000FF10FF141414FF141010101F0000000085
:102FA000F010FFFFFFFFFFF0F0F0F0F0FFFFFF0079
:102FB00000000000FFFF0F0F0F0F0F38444438448C
:102FC0007C2A2A3E147E02020606027E027E0263EC
:102FD000554941633844443C04407E201E2006028B
:102FE0007E020299A5E7A5991C2A492A1C4C720168
:102FF000724C304A4D4D303048784830BC625A46A9
:103000003D3E494949007E0101017E2A2A2A2A2A99
:1030100044445F444440514A444040444A51400083
:1030200000FF0103E080FF000008086B6B08361208
:10303000362436060F090F0600001818000000108D
:1030400010003040FF0101001F01011E00191D1773
:1030500012003C3C3C3C000000000000000000244A
:103060000027002A0000000000250028002B000097
:1030700000000023002600290004040404040404C2
:103080000402020202020203030303030301020417
:1030900008102040800102040810200102040810DA
:1030A00020AED5F0A83FD300408D14A1C8DA12811C
:1030B000CFD9F1DB40A4A6AF200021007F2200077A
:1030C000506C656173652077616974004144433ACF
:1030D000200074656D703A2000536574206D656141
:1030E000737572656400537465703A2000FFFFFFCA
:1030F000FFFFFF8003867080038003867080039F3C
:10310000F3E1309FF39FF3E1309FF3983301CC98C4
:1031100033983301CC9833983387C098339833E190
:10312000C098339833E1C098339FF398C09FF39FC2
:10313000F398C09FF3800366CC8003800366CC8045
:1031400003FFFF010CFFFFFFFF01001FFF81006174
:10315000301F3F873CE6FC8733873CE6FC87F3F86B
:10316000039E0F1F03F8039E0F1F03E13CFE0C0795
:10317000CFE13CFE0C07CF99033E3086C3E6CF3843
:103180000F9EF3E6CF380F9EF39E0327CC81039E5C
:103190000327CC8103E0FFE10CE6CFE0FFE10CE682
:1031A000CF9803060000FF9803060000FFFFFF1EF4
:1031B000F0F8038003663099C38003663099C39F9B
:1031C000F3010CF8FF9FF3010CF8FF9833393C0131
:1031D000CF9833393C01CF9833FF0C793F98333E79
:1031E000CCE0F398333ECCE0F39FF33E0098CF9FC2
:1031F000F33E0098CF80033E30E7C380033E30E7C4
:10320000C3FFFFFFFFFFFFFFFFFFFFFFFF30303077
:103210000076312E364C31005600560043000080B7
:103220000080018001800380078007F00FF00FE02D
:103230001FC001C00180018001800100010012480F
:1032400012481FF8E0072E142C04E807200420047D
:10325000E00720042814E0071FF8124812484552DE
:10326000524F5200484F4C44004845415400574F7C
:10327000524B5900424F4F535400534C4545500058
:103280004F46460000007E007F00738061C061E011
:1032900073F03FF81FFC0FFE07FF03FF01FE00FC69
:1032A000007800300102040810204080000000086F
:1032B00000020100000304070000000000000000FD
:1032C0001D2FC03811241FBECFEFD8E0DEBFCDBF09
:1032D00012E0A0E0B1E0EEE7FCE702C005900D923D
:1032E000A237B107D9F727E0A2E7B2E001C01D92EB
:1032F000A53CB207E1F719E1C1E6D9E104C0219785
:10330000FE010E94353CC036D107C9F70E94E12F6B
:103310000C94323E0C9400004F925F926F927F9219
:103320008F929F92AF92BF92CF92DF92EF92FF92D5
:103330000F931F93CF93DF9300D000D0CDB7DEB7AC
:103340004B015C0129013A016701780120E030E07E
:10335000A9010E943A3987FDA6C020E030E0A9010A
:10336000C301B2010E943A3987FD9DC020E030E0E0
:10337000A901C801B6010E943A3987FD94C081E0D5
:1033800020918507309186072130310509F080E0D2
:103390008093A60780926B0790926C07A0926D07AE
:1033A000B0926E0740926F0750927007609271075B
:1033B00070927207C0927307D0927407E0927507FB
:1033C000F09276076091990770919A0780919B0718
:1033D00090919C070E943F3920E030E04AE754E496
:1033E0000E94733B69837A838B839C8380927707E7
:1033F00090927807A0927907B0927A079B01AC016E
:10340000C301B2010E94A0392B013C0140927B070D
:1034100050927C0760927D0770927E0729813A81E5
:103420004B815C81C701B6010E94733B6B017C013B
:10343000C0927F07D0928007E0928107F0928207C6
:103440008091830790918407019769F5A501940104
:1034500060E070E0CB010E94063B609377077093B9
:1034600078078093790790937A07A301920160E02F
:1034700070E0CB010E94063B60937B0770937C0752
:1034800080937D0790937E07A701960160E070E02E
:10349000CB010E94063B60937F0770938007809367
:1034A0008107909382070F900F900F900F90DF91FC
:1034B000CF911F910F91FF90EF90DF90CF90BF9031
:1034C000AF909F908F907F906F905F904F900895F6
:1034D00080389105B0F46034710598F4E4EAF2E3C1
:1034E00090E1969FD001A0781124A80F6770E60F95
:1034F000F11D9491AE53BD4F442321F08C91982B34
:103500009C93089590958C919823FACFDF92EF9237
:10351000FF920F931F93CF93DF937C01EB01D22E89
:103520008B01040F111DC8010134110514F080E452
:1035300090E0C817D9073CF44D2DBE01C7010E9489
:10354000681A2196F0CFDF91CF911F910F91FF90D4
:10355000EF90DF900895CF92DF92EF92FF920F935A
:103560001F93CF93DF936B01122FEC017C01E40ECC
:10357000F11CCE15DF0544F4202F412FB601CE01FA
:103580000E94861A2196F5CFDF91CF911F910F915E
:10359000FF90EF90DF90CF9008952F923F924F923F
:1035A0005F926F927F928F929F92AF92BF92CF92D3
:1035B000DF92EF92FF920F931F93CF93DF9300D090
:1035C0001F92CDB7DEB7C22ED12C9601280F391F1E
:1035D00037FD4FC0803891050CF04BC0E9824A019D
:1035E0007B013C01402E512C160127E0220E311C9C
:1035F00093E0359427949A95E1F78B01B12CA12C97
:103600001B821A82EA81FB8183E0F595E7958A9512
:10361000E1F7EA0DFB1DE80DF91DE4918A819B811C
:103620008770992720E830E002C0359527958A9564
:10363000E2F7C901F0E0E223F923EF2B41F04981E1
:10364000B8018A819B81860D971D0E94681A8A8124
:103650009B8101969B838A838C159D059CF2A20C0D
:10366000B31C0F5F1F4FC8018E199F098415950564
:103670003CF20F900F900F90DF91CF911F910F911F
:10368000FF90EF90DF90CF90BF90AF909F908F9082
:103690007F906F905F904F903F902F90089580E0C3
:1036A000E2ECF2E081118FEF00248193819381930A
:1036B00081930394D1F7EDEAF7E017861686158615
:1036C000148608950895AF92BF92CF92DF92EF9241
:1036D000FF920F931F93CF93DF936C017B018B01BC
:1036E000040F151FEB015E01AE18BF08C017D1070C
:1036F00059F06991D601ED91FC910190F081E02D96
:10370000C6010995892B79F7C501DF91CF911F91EA
:103710000F91FF90EF90DF90CF90BF90AF90089502
:10372000FC01538D448D252F30E0842F90E0821BC7
:10373000930B541710F0CF96089501970895FC014C
:10374000918D828D981761F0A28DAE0FBF2FB11DA4
:103750005D968C91928D9F5F9F73928F90E00895FC
:103760008FEF9FEF0895FC01918D828D981731F0B6
:10377000828DE80FF11D858D90E008958FEF9FEF0A
:103780000895FC01918D228D892F90E0805C9F4FE0
:10379000821B91098F739927089582EC96E00E940D
:1037A000C11B21E0892B09F420E0822F089580E0DD
:1037B00090E0892B29F00E94CD1B81110C94000010
:1037C0000895FC01A48DA80FB92FB11DA35ABF4FB6
:1037D0002C91848D90E001968F739927848FA68910
:1037E000B7892C93A089B1898C91837080648C9364
:1037F000938D848D981306C00288F389E02D808113
:103800008F7D80830895EF92FF920F931F93CF9344
:10381000DF93EC0181E0888F9B8D8C8D98131AC00B
:10382000E889F989808185FF15C09FB7F894EE89F2
:10383000FF896083E889F98980818370806480834F
:103840009FBF81E090E0DF91CF911F910F91FF909A
:10385000EF900895F62E0B8D10E00F5F1F4F0F7342
:103860001127E02E8C8D8E110CC00FB607FCFACFFD
:10387000E889F989808185FFF5CFCE010E94E11B9F
:10388000F1CFEB8DEC0FFD2FF11DE35AFF4FF082CE
:103890009FB7F8940B8FEA89FB8980818062CFCF34
:1038A000CF93DF93EC01888D8823B9F0AA89BB8977
:1038B000E889F9898C9185FD03C0808186FD0DC062
:1038C0000FB607FCF7CF8C9185FFF2CF808185FF83
:1038D000EDCFCE010E94E11BE9CFDF91CF9108959A
:1038E000833081F028F4813099F08230A9F0089576
:1038F0008730A9F08830C9F08430B1F4809180001D
:103900008F7D03C0809180008F7780938000089521
:1039100084B58F7784BD089584B58F7DFBCF80916A
:10392000B0008F778093B00008958091B0008F7DB4
:10393000F9CFCF93DF93282F30E0F901E455FD4C08
:103940008491F901E357FF4CD491F901E758FF4CFA
:10395000C491CC23A1F081110E94701CEC2FF0E0E7
:10396000EE0FFF1FE159FF4CA591B491EC91ED23AF
:1039700081E090E009F480E0DF91CF91089580E04C
:1039800090E0FACF1F93CF93DF93282F30E0F90117
:10399000E455FD4C8491F901E357FF4CD491F901B2
:1039A000E758FF4CC491CC23A9F0162F81110E9437
:1039B000701CEC2FF0E0EE0FFF1FEB59FF4CA591B0
:1039C000B4918FB7F894EC91111108C0D095DE2313
:1039D000DC938FBFDF91CF911F910895DE2BF8CF3D
:1039E000CF93DF9390E0FC01E357FF4C249187587D
:1039F0009F4CFC0184918823C9F090E0880F991FA7
:103A0000FC01E55AFF4CA591B491FC01EB59FF4C28
:103A1000C591D49161110DC09FB7F8948C912095F8
:103A200082238C938881282328839FBFDF91CF91A5
:103A30000895623051F49FB7F8943C91822F80959D
:103A400083238C93E8812E2BEFCF8FB7F894EC91E2
:103A50002E2B2C938FBFEACFCF93DF93EC0161E045
:103A600089E00E94F01C209731F460E089E0DF914A
:103A7000CF910C94C21CCF3FD10511F461E0F6CF79
:103A8000E5EBF2E3E491E33029F140F4E130B1F009
:103A9000E230D9F0C038D1058CF7E7CFE73021F11B
:103AA000E83051F1E430B1F780918000806280937A
:103AB0008000D0938B00C0938A0004C084B58068D6
:103AC00084BDC7BDDF91CF91089584B5806284BD68
:103AD000C8BDF8CF80918000806880938000D0932B
:103AE0008900C0938800EECF8091B00080688093F9
:103AF000B000C093B300E6CF8091B00080628093A5
:103B0000B000C093B400DECF3FB7F89480918B0231
:103B100090918C02A0918D02B0918E0226B5A89B47
:103B200005C02F3F19F00196A11DB11D3FBFBA2F4F
:103B3000A92F982F8827BC01CD01620F711D811D0F
:103B4000911D42E0660F771F881F991F4A95D1F794
:103B500008958F929F92AF92BF92CF92DF92EF9291
:103B6000FF924B015C010E94841D6B017C010E944D
:103B7000841D6C197D098E099F09683E734081057B
:103B80009105A8F321E0821A9108A108B10888EEF6
:103B9000C80E83E0D81EE11CF11C81149104A1041D
:103BA000B10429F7FF90EF90DF90CF90BF90AF90D6
:103BB0009F908F9008952FB7F8946091870270912D
:103BC00088028091890290918A022FBF089584E92A
:103BD0008093BC008091BC0084FDFCCF089580934D
:103BE000BB0084E88093BC008091BC0087FFFCCFC1
:103BF000089584EA8093BC008091BC0087FFFCCFCD
:103C000088E70C94EF1D0E94F91D80E48093BB00AF
:103C100084E88093BC00E2ECF2E09091BC0097FF56
:103C2000FCCF91919093BB008093BC0096E0E23C66
:103C3000F90799F78091BC0087FFFCCF0C94E71D32
:103C4000CF93C82F0E94F91D80E00E94EF1D8C2F9A
:103C50000E94EF1DCF910C94E71D480F592F511D65
:103C60004138510514F040E850E0481BFB0177FD56
:103C7000379633E0F595E7953A95E1F7F695FE2FFF
:103C8000EE27F795E795E80FF91FEE53FD4F6770A4
:103C9000772781E090E001C0880F6A95EAF7382F16
:103CA000213041F4415078F08191DF011197832B4D
:103CB0008C93F8CF8095415030F09191DF011197AE
:103CC00098239C93F8CF0895CF92DF92EF92FF92C2
:103CD0000F93CF93DF936C017B01C42FD22F202F42
:103CE0000E942D1EB7016D0F711D61507109603466
:103CF00071052CF4202F4C2FC6010E942D1E202F61
:103D00004D2FB701C6010E94861AC6018C0F911D66
:103D1000202F4D2FB7010197DF91CF910F91FF9089
:103D2000EF90DF90CF900C94861A2F923F924F9293
:103D30005F926F927F928F929F92AF92BF92CF923B
:103D4000DF92EF92FF920F931F93CF93DF93CDB744
:103D5000DEB72A970FB6F894DEBF0FBECDBF9A83A9
:103D600089836A3061F5DC0152968C91B8E08B9FB3
:103D700090011124E981FA8186859785820F931F2E
:103D8000978786871586148681E090E02A960FB67D
:103D9000F894DEBF0FBECDBFDF91CF911F910F9181
:103DA000FF90EF90DF90CF90BF90AF909F908F905B
:103DB0007F906F905F904F903F902F9008956D305F
:103DC00019F329813A813A872987D9011C96AD9048
:103DD000BC90B0E8AB16B1040CF07BC0F901C6840E
:103DE000D784F0E4CF16D1040CF073C0D9015296F9
:103DF0006C90529745E09501649E200D311D112471
:103E0000121613060CF065C0262C312C910153E0DC
:103E1000220F331F5A95E1F72C0D3D1D1216130684
:103E20000CF057C05196BC91BB83E985FA85F089A7
:103E3000FC83649FB00111249B01255A344D3A83C1
:103E40002983712CE981FA818491F5E07F1201C008
:103E500080E0460138E0532E282F30E03E832D834A
:103E60004C8080FF4B80411004C03B818C8138170F
:103E7000E1F010E000E00615C0F4D501A00FB11F7D
:103E8000B887AF83F12CE12CE61460F4B701680D1C
:103E9000791D442D8F8198850E94681ABFEFEB1A17
:103EA000FB0AF2CF0F5F1F4FE6CF8D819E81959564
:103EB00087955A94820C931C5110CECF7394E9814C
:103EC000FA813196FA83E983A20CB31CF6E07F12E3
:103ED000B9CFA985BA8552962C915297422F50E0BE
:103EE0001C968D919C91B6E02B9F800D911D112405
:103EF000E985FA85958784872389222309F444CFAD
:103F00006AEF64039001659F300D112420583F4FE4
:103F1000281739070CF038CFDF010190F081E02D30
:103F20000190F081E02D6AE0CD0109952DCF0F932E
:103F30001F93CF93DF938C01D0E0C0E0F801EC0F2A
:103F4000FD1F6491662341F08DEA97E00E94951E63
:103F5000892B11F02196F2CFCE01DF91CF911F91E5
:103F60000F910895682F8DEA97E00C94951E90E0CC
:103F700080E0089580917A00806980937A008EE4D1
:103F800080937C0061E070E080E090E00E94A91DD9
:103F900083B7817F826083BF80E130E020E093B708
:103FA000916093BF889593B79E7F93BF90917A005D
:103FB00096FDFCCF4091780050917900240F351F79
:103FC000815069F780917A008F7780937A0084E03E
:103FD000369527958A95E1F750E040E064EB7BE267
:103FE00081E190E00E94743AC901089580917A00BD
:103FF000806980937A0088EC80937C0064E170E0B3
:1040000080E090E00E94A91D83B7817F826083BF1A
:1040100080E270E060E093B7916093BF889593B7BA
:104020009E7F93BF90917A0096FDFCCF20917800FF
:1040300030917900620F731F815069F780917A0087
:104040008F7780937A00769567957695679562521B
:104050007A4090E080E00E943F3926EF38E24CE160
:1040600051E40E94733B089590917A009069909377
:104070007A008E50806480937C0083B7817F826059
:1040800083BF20E290E080E033B7316033BF889592
:1040900033B73E7F33BF30917A0036FDFCCF40917D
:1040A000780050917900840F951F215069F7209175
:1040B0007A002F7720937A0025E0969587952A95A8
:1040C000E1F708958FE00E943420A0919202B09110
:1040D00093029C010E94F73A0E94413928E539E792
:1040E00043E353E40E94733B0E94EC3BCB010895F1
:1040F0002091A00230E0EDE1F2E090E080E0AF013D
:104100004D5152404217530724F44191840F911DA1
:10411000F6CF089580919902882369F086E00E9485
:10412000991C892B41F06AE070E080E090E00E94E9
:10413000A91D1092990208950F931F93CF93809118
:104140004801882399F0CFEF0FEE11E061E085E0A0
:104150000E94C21CC8010197F1F760E085E00E944F
:10416000C21CC8010197F1F7C15081F7CF911F918F
:104170000F9108952F923F924F925F926F927F928C
:104180008F929F92AF92BF92CF92DF92EF92FF9267
:104190000F931F93CF93DF9310E000E0D0E0C0E0D7
:1041A0003EE3E32EF12C40ECC42ED12CAA24A394A0
:1041B000B12C60E2662E712C70E4272E312C4C2E2F
:1041C00086E00E94991C21E0892B09F020E02093D1
:1041D0009902F0929F02E0929E02D0929D02C092BC
:1041E0009C02B0929B02A0929A0282E890E0909387
:1041F000AB028093AA028091AA029091AB0295959E
:104200008795582E9FE1591243C0F0929F02E09289
:104210009E02D0929D02C0929C02B0929B02A092FC
:104220009A02EEEBF0E0F093AB02E093AA029FE576
:10423000592E0E944F1B82E08093BF071093BA074C
:104240000093B907E0E3F0E0F093BC07E093BB070D
:104250008EE50E94B21F1092BA071092B9077092B1
:10426000BC076092BB07912C812C841438F5809197
:10427000BE02F40196E0989FE00DF11D1124E15B70
:10428000FE4F80810E94B21FEFEF8E1A9E0AEDCF83
:10429000F0E65F12CECFF0929F02E0929E02D092A3
:1042A0009D02C0929C02B0929B02A0929A02309210
:1042B000AB022092AA0280E2582EBBCF1093BA071D
:1042C0000093B9077092BC076092BB07852D0E94CE
:1042D000B21F0E948A200E94031E86E00E94991C41
:1042E000892B09F088CF80919902811184CF809029
:1042F000BE02F6E08F9E40011124C401815B9E4FF7
:104300004C01FC01EC0FFD1F50820E949C206AE0D2
:1043100070E080E090E00E94A91D2196005F1F4F91
:10432000C530D10509F04BCFF4011582DF91CF9153
:104330001F910F91FF90EF90DF90CF90BF90AF90C3
:104340009F908F907F906F905F904F903F902F90B5
:1043500008952F923F924F925F926F927F928F9229
:104360009F92AF92BF92CF92DF92EF92FF920F9304
:104370001F93CF93DF93982EE091A002F0E0E35ECD
:10438000FD4F80818150990B10929F0210929E02E6
:10439000880F991F90939D0280939C0281E090E08A
:1043A00090939B0280939A02892D90E0880F991F29
:1043B0009093AB028093AA0286E00E94991C21E0B0
:1043C000892B09F020E0209399021092BE0781E02A
:1043D0008093BD0738E3F32E41E3242E312CA090C7
:1043E000AA02B090AB02B594A7941A2D6501DD2402
:1043F000960129193109F29EC001F39E900D1124F6
:10440000C80FD91F209709F1662777276C1B7D0BF2
:10441000072E000C880B990B0E94413920E030E0F8
:1044200040E05FE30E94A0392B013C01BE01DD0F9B
:10443000880B990B0E9441399B01AC01C301B20169
:104440000E94073B0E94E53BEB010E944F1B460187
:1044500082E0881A91083E01260193E0490E511C22
:1044600097FC20C0E091A002F0E0E35EFD4F808168
:1044700088151904B9F0B4F00E947820F401E80F0F
:10448000F11DEE0FFF1FEF52FE4F40815181EE24D0
:10449000E39400E320E370E060E0C30188549109F5
:1044A0000E94CD1A8FEF881A980A98E3690E711C42
:1044B00048145904A9F68091BA0281113AC00E94A9
:1044C0007820F601E80FF11DEE0FFF1FEB57FE4FAE
:1044D00040815181EE24E39400E124E260E370E046
:1044E00080E390E00E94CD1A0E94031E0E948A2061
:1044F00086E00E94991C892BD1F480919902811148
:1045000016C00E949C20812FDF91CF911F910F91A7
:10451000FF90EF90DF90CF90BF90AF909F908F90E3
:104520007F906F905F904F903F902F9008959A2CBE
:1045300056CF80E390E09093BA078093B90730920A
:10454000BC072092BB0781E08093BF070E947820C0
:104550008A0D863208F0A0C0E82FF0E0EE54FD4D41
:104560000C94353CD822DD22E022E322E622E92227
:10457000EC22EF22F222F522F822FB22FE22012376
:10458000042307230A230D2310231323162319239F
:104590001C231F232223252328232B232E233123CF
:1045A000342337233A233D234023432346234923FF
:1045B0008AE49BE20E94971F97CF85E49BE2FACFA3
:1045C0008FE39BE2F7CF87E39BE2F4CF80E39BE2AC
:1045D000F1CF89E29BE2EECF84E29BE2EBCF8EE16A
:1045E0009BE2E8CF87E19BE2E5CF80E19BE2E2CF6F
:1045F00086E09BE2DFCF8FEF9AE2DCCF88EF9AE292
:10460000D9CF84EF9AE2D6CF8FEE9AE2D3CF87EE5E
:104610009AE2D0CF81EE9AE2CDCF8BED9AE2CACF6B
:1046200086ED9AE2C7CF80ED9AE2C4CF8CEC9AE295
:10463000C1CF86EC9AE2BECF81EC9AE2BBCF8AEB87
:104640009AE2B8CF86EB9AE2B5CF82EB9AE2B2CF8C
:104650008CEA9AE2AFCF88EA9AE2ACCF85EA9AE296
:10466000A9CF82EA9AE2A6CF8EE99AE2A3CF8BE99C
:104670009AE2A0CF88E99AE29DCF85E99AE29ACFA3
:1046800082E99AE297CF86E89AE294CF81E89AE2AB
:1046900091CF8CE79AE28ECF88E79AE28BCF3F9258
:1046A0004F925F926F927F928F929F92AF92BF9242
:1046B000CF92DF92EF92FF920F931F93CF93DF93EE
:1046C000CDB7DEB72E970FB6F894DEBF0FBECDBFC5
:1046D0008091BD02882309F4A5C110925F07109252
:1046E0006007109261071092620780905F079090B8
:1046F0006007A0906107B0906207C090B302D090AD
:10470000B402E090B502F090B602A7019601C5018F
:10471000B4010E94063B2B013C0120E030E0A901DE
:104720000E941B3C18160CF0A0C1C301B2010E94EC
:10473000EC3B80914901882309F4B8C1C092670716
:10474000D0926807E0926907F0926A07E12CF12C99
:1047500000EA10E420E030E040E450E46E317105FE
:1047600040F0E12CF12C00E81FE320E030E040E0D5
:104770005FE360E070E080E391E40E948C19809137
:10478000A507882309F42AC10E94DB1D6D837E835F
:104790008F83988780918D0790918E07A0918F07C6
:1047A000B09190074D815E816F817885481B590BD0
:1047B0006A0B7B0B8091990790919A07A0919B07B8
:1047C000B0919C07481759076A077B0708F406C190
:1047D000E0918707F091880780819181A281B38160
:1047E00089839A83AB83BC83E0918B07F0918C071C
:1047F0009C01AD0160817181828193810E94063BA1
:104800004B015C01209195073091960740919707E5
:104810005091980769817A818B819C810E94063B27
:104820006B017C0120917B0730917C0740917D07D3
:1048300050917E07C501B4010E94A03920919107D3
:104840003091920740919307509194070E94073B43
:104850002B013C014092910750929207609293077E
:10486000709294073090A60731101AC020917707F4
:10487000309178074091790750917A07C701B601C6
:104880000E94A0399B01AC01C301B2010E94063B0A
:104890006093910770939207809393079093940786
:1048A0004090910750909207609093077090940702
:1048B0001091A1079091A2079E87A091A307AD87B1
:1048C0000091A407212F392F4A2F502FC301B20185
:1048D0000E941B3C18160CF0CCC0812F9E85AD8524
:1048E000B02F8093910790939207A0939307B09372
:1048F0009407332009F4D6C02091770730917807C8
:104900004091790750917A07C501B4010E94A039FE
:104910004B015C0120917F07309180074091810716
:1049200050918207C701B6010E94A0399B01AC01DA
:1049300060919107709192078091930790919407ED
:104940000E94063BA50194010E94073B6B017C017C
:104950009B01AC01612F7E858D85902F0E943A3995
:1049600087FD18C010919D0790919E079E87A0918A
:104970009F07AD870091A007212F392F4A2F502F75
:10498000B601C7010E943A3987FD04C01C2DDE869E
:10499000ED860F2DE0918907F0918A07812F9E8582
:1049A000AD85B02F80839183A283B38389819A815F
:1049B000AB81BC818093950790939607A09397074E
:1049C000B09398078D819E81AF81B88580938D07C4
:1049D00090938E07A0938F07B09390076091630721
:1049E0007091640780916507909166070E94E53B8E
:1049F000CB012E960FB6F894DEBF0FBECDBFDF9170
:104A0000CF911F910F91FF90EF90DF90CF90BF90CB
:104A1000AF909F908F907F906F905F904F903F905E
:104A20000C942C1D8091BC02609144017091450151
:104A300081110EC08091B1029091B2022091BB020F
:104A4000BC01222329F060914301680F792F711D69
:104A500090E080E00E943F3960935F0770936007A9
:104A6000809361079093620740CEC301B2019058D2
:104A70005ECE80919D0790919E07A0919F07B09177
:104A8000A00789879A87AB87BC879C01AD01C301CA
:104A9000B2010E943A3987FF2CCF89859A85AB8570
:104AA000BC851FCF812C912C540134CF20E030E005
:104AB00040E05FE3C701B6010E94073B9B01AC01E8
:104AC000C501B4010E941B3C18164CF410926307F8
:104AD0001092640710926507109266077FCF80E0FE
:104AE00090E0AFE7B3E48093630790936407A093EB
:104AF0006507B093660772CF4F925F926F927F9275
:104B00008F929F92AF92BF92CF92DF92EF92FF92DD
:104B1000CF93DF938090940290909502A09096029C
:104B2000B0909702C091BE02D0E0C501B4010E94CE
:104B3000E53B6B017C0120E030E048E453E4C50133
:104B4000B4010E943A3993E0CC0FDD1F9A95E1F74A
:104B5000CE5FDE4F87FF31C02881398150E040E0D1
:104B60002551310941095109C701B6010E94253C6F
:104B700028EC30E040E050E00E94743ACA01B901EC
:104B80006B5E7F4F8F4F9F4F0E9441396093B302FE
:104B90007093B4028093B5029093B602DF91CF91E7
:104BA000FF90EF90DF90CF90BF90AF909F908F904D
:104BB0007F906F905F904F9008954A805B80712C3A
:104BC000612C20E030E04CE853E4C501B4010E94C0
:104BD0003A3987FF1FC088809980B12CA12CA7018A
:104BE0009601285C310941095109C301B2016819D4
:104BF00079098A099B090E94253C20E530E040E0C4
:104C000050E00E94743ACA01B901680D791D8A1DED
:104C10009B1DBACF2C813D8150E040E0241935091D
:104C200046095709C701B6016851714081099109C8
:104C30000E94253C20E530E040E050E00E94743ABC
:104C4000CA01B901640D751D861D971D9DCFFC011C
:104C500001900020E9F73197AF01481B590BBC01C7
:104C60008DEA97E00C94631B8F929F92AF92BF9254
:104C70000F931F93CF93DF93CDB7DEB7A1970FB6F6
:104C8000F894DEBF0FBECDBF19A2423008F44AE04F
:104C90008E010F5D1F4F842E912CB12CA12CA501EC
:104CA00094010E94D53AE62FB901CA01EA30F4F422
:104CB000E05DD801EE938D01232B242B252B79F772
:104CC00090E080E0109719F0CD010E942726A19670
:104CD0000FB6F894DEBF0FBECDBFDF91CF911F910D
:104CE0000F91BF90AF909F908F900895E95CE1CFB6
:104CF000CF92DF92EF92FF92CF93DF9397FF19C08D
:104D00006B017C018DE20E94B21FEC0166277727C0
:104D1000CB016C197D098E099F094AE00E94342657
:104D20008C0F9D1FDF91CF91FF90EF90DF90CF9080
:104D300008954AE0DF91CF91FF90EF90DF90CF9000
:104D40000C9434264F925F926F927F928F929F9233
:104D5000AF92BF92CF92DF92EF92FF920F931F9389
:104D6000CF936B017C01742EAC019B010E94203C0F
:104D7000882399F082E692E0CF911F910F91FF90E6
:104D8000EF90DF90CF90BF90AF909F908F907F90EB
:104D90006F905F904F900C94272646015701E8943E
:104DA000B7F82FEF3FEF4FE75FE7C501B4010E946F
:104DB000203C81110DC02FEF3FEF4FE75FE7C501AA
:104DC000B4010E943A3918161CF486E692E0D4CF5A
:104DD0002FEF3FEF4FE75FE4C701B6010E941B3C96
:104DE00018161CF48AE692E0C7CF2FEF3FEF4FE78B
:104DF0005FECC701B6010E943A3987FDF3CF20E08E
:104E000030E0A901C701B6010E943A3910E000E084
:104E100087FF08C08DE20E94B21F8C01F7FAF09460
:104E2000F7F8F094C0E060E070E080E09FE37C166B
:104E300041F020E030E040E251E40E94733BCF5F5C
:104E4000F6CFA70196010E94073B2B013C010E946F
:104E5000EC3B4B015C014AE00E9434267C01E00EF1
:104E6000F11ECC23B1F1C501B4010E943F399B0171
:104E7000AC01C301B2010E94063B4B015C018EE212
:104E80000E94B21FE80EF91EC15018F120E030E078
:104E900040E251E4C501B4010E94A0392B013C015C
:104EA0000E94EC3B4B01B12CA12C4AE0C501B4019E
:104EB0000E943426E80EF91EC501B4010E943F3954
:104EC0009B01AC01C301B2010E94063B4B015C0196
:104ED000DBCFC701CF911F910F91FF90EF90DF9033
:104EE000CF90BF90AF909F908F907F906F905F908A
:104EF0004F900895CF92DF92EF92FF920F931F93FE
:104F0000CF93DF93C82F81E0DC2FD827D093BE0743
:104F1000C093BD078093BF070C2F2EE046E661E3E8
:104F200070E081E090E00E94641E2091BF02309109
:104F3000C002253F81E03807B8F4A4E6B0E00E9443
:104F4000F73A24EF31E040E050E00E94743ABA01B1
:104F5000A9014E5F5F4F6F4F7F4F2EE061E370E01E
:104F600081E090E00E94AB1A60915F07709160074A
:104F700080916107909162070E94E53B9B01AC0123
:104F8000A4E6B0E00E94933A34EFC32EDD24D3941C
:104F9000E12CF12CA70196010E94743ADA01C901B3
:104FA0000296A11DB11D02970C2F2DE043E062E394
:104FB00070E00E94AB1A60915F077091600780916A
:104FC0006107909162070E94E53B9B01AC01A4E65A
:104FD000B0E00E94933AA70196010E94743ADA0168
:104FE000C9010296A11DB11D039724E045E06CE3C1
:104FF00070E00E94AB1A60915F077091600780912A
:105000006107909162070E94E53B9B01AC01A4E619
:10501000B0E00E94933AA70196010E94743A890178
:105020009A010E5F1F4F2F4F3F4F0150110941E36F
:10503000E42EF12C4D2FB701C8010E94681A8FEFA2
:10504000E81AF80A8DE3E816F104A1F760915F070A
:105050007091600780916107909162070E94E53B23
:105060009B01AC01A4E6B0E00E94933A24EF31E04A
:1050700040E050E00E94743ADA01C9010296A11D95
:10508000B11D0397ED2E04E025E044E75AE26BE3FF
:1050900070E00E94CD1A0C2F2EE047E161E370E032
:1050A00088E690E00E94641E609163077091640737
:1050B00080916507909166070E94E53B9B01AC01DA
:1050C0002F5F310941095109A7E1B0E00E94933AED
:1050D000CC24C394DD24DA94ED2CFD2CA701960199
:1050E0000E94743A422F2EE061E370E088E690E07F
:1050F0000E94AB1AC093BE07D093BD0782E090E038
:105100009093BA078093B90707E310E01093BC07A8
:105110000093BB0760915F07709160078091610702
:105120009091620740E00E94A22688EF0E94B21F81
:1051300082E79AE20E94971F89E690E09093BA076F
:105140008093B9071093BC070093BB076091630776
:105150007091640780916507909166070E94E53B16
:105160009B01AC012F5F310941095109A4E6B0E070
:105170000E94933AA70196010E94743ACA01B901AC
:105180000E94782680E79AE20E94971FD093BE077C
:10519000C093BD07DF91CF911F910F91FF90EF90CA
:1051A000DF90CF9008956F927F928F929F92AF92EF
:1051B000BF92CF92DF92EF92FF920F931F93CF9304
:1051C000DF93B090BE0277247394B11001C0712CAC
:1051D000809142018150990B10929F0210929E0281
:1051E000880F991F90939D0280939C0281E090E02C
:1051F00090939B0280939A028B2D90E0880F991FC9
:105200009093AB028093AA0286E00E94991C21E051
:10521000892B09F020E020939902FF24F39472E097
:10522000972EE6E08E2EFCE0CF2ED12C0E944F1B55
:10523000C091AA02D091AB02D595C795EC2E8E01F4
:105240001127C801870D911D77FC9A958B1991093B
:10525000712C97FD06C08330910514F082E090E038
:10526000782EF092BE071092BD079092BF07109261
:10527000BA071092B9071092BC071092BB0780E5DD
:105280009BE20E94971F1092BE07F092BD071092FA
:10529000BA071092B907A72C072C000CBB08C50150
:1052A000019654E0880F991F5A95E1F79093BC0737
:1052B0008093BB078EE49BE20E94971F6C2E6718B9
:1052C00090E080E098012A193B09590120914201A0
:1052D0008C010F5F1F4F6216D0F4D092BA07C092B4
:1052E000B907980144E0220F331F4A95E1F7309344
:1052F000BC072093BB078A0D9B1D889E9001899E49
:10530000300D1124C901815B9E4F0E942726C801E0
:10531000639403301105D1F60E948A200E94031E77
:1053200086E00E94991C892BB9F480919902811121
:1053300013C00E949C20E092BE02DF91CF911F918A
:105340000F91FF90EF90DF90CF90BF90AF909F9024
:105350008F907F906F900895BC2E68CF0E941D3E65
:10536000EF92FF920F931F93CF93DF93EC017B019A
:105370008A0188819981009729F02A813B8124172D
:10538000350788F4B8016F5F7F4F0E94603D00973A
:1053900091F0998388831B830A832C813D81232B81
:1053A00011F4FC0110821D830C83B701888199815F
:1053B0000E942B3E0CC088819981009711F00E94B9
:1053C000D73C198218821D821C821B821A82CE0150
:1053D000DF91CF911F910F91FF90EF9008951F9350
:1053E000CF93DF93EC01162F0E945E3A181739F025
:1053F000612FCE01DF91CF911F910C94663ADF911E
:10540000CF911F910895AF92BF92CF92DF92EF920A
:10541000FF920F931F93CF93DF936091470182E038
:1054200090E00E94EF296091460183E090E00E94A5
:10543000EF296091450184E090E00E94EF2960919E
:10544000440185E090E00E94EF296091430186E0ED
:1054500090E00E94EF2960914C0187E090E00E946B
:10546000EF2960914B0188E090E00E94EF29609164
:105470004A0189E090E00E94EF296091C1028AE030
:1054800090E00E94EF29609149018BE090E00E943A
:10549000EF29609148018CE090E00E94EF29609133
:1054A000BE028DE090E00E94EF29609142018EE003
:1054B00090E00E94EF296091BA028FE090E00E9494
:1054C000EF296091980280E190E00E94EF2981E14C
:1054D000E82EF12C10E006E0809142011817B8F593
:1054E000109F60011124D0E0C0E0FE01EC0DFD1D15
:1054F000E15BFE4F6081C7018C0F9D1F0E94EF2969
:105500002196C630D10589F7670186E0C80ED11C07
:1055100088E0189FE0011124CE5FDE4F8EE0E80E98
:10552000F11C69812296C6010E94EF29560182E092
:10553000A80EB11CFE0132976081C60101960E943F
:10554000EF296501AE14BF0461F71F5FC5CFDF917E
:10555000CF911F910F91FF90EF90DF90CF90BF9070
:10556000AF9008958F929F92AF92BF92CF92DF92A9
:10557000EF92FF92CF938FEF90E00E942C1D8BEA69
:1055800094E00197F1F78EE00E9434207C018AE0DC
:105590000E94991C90917202981729F091E09093C3
:1055A000B70280937202809101019FEF980F909350
:1055B0000101811106C00E9462209093B90280937C
:1055C000B8026091630770916407809165079091BC
:1055D00066070E94E53BCB010E942C1D809094023F
:1055E00090909502A0909602B0909702B70190E03B
:1055F00080E00E943F39A50194010E94063B2DECFA
:105600003CEC4CE45DE30E94A039A50194010E94AA
:10561000073B609394027093950280939602909357
:1056200097020E947C256091BF027091C00290E0B9
:1056300080E00E943F396B017C0120915F0730912F
:10564000600740916107509162070E943A398111C9
:10565000B5C02091B3023091B4024091B50250918F
:10566000B602C701B6010E94063B6B017C0120E037
:1056700030E0A9010E941B3C18160CF095C020E0F8
:1056800030E040EA50E4C701B6010E941B3C181606
:105690000CF494C06091B1027091B20290E080E08D
:1056A0000E943F392091B3023091B4024091B5027B
:1056B0005091B6020E94063B6B017C0120E030E075
:1056C000A9010E941B3C18160CF087C0C701B60147
:1056D0000E94EC3B6530710508F083C080914E015B
:1056E000811105C080914D0181110E949C2081E0B3
:1056F00080934E0110924D018091BF029091C002A3
:10570000853F21E0920710F01092000120910001E6
:10571000211140C0843F9140E8F58FEF90E00E9456
:105720002C1D0E949C20C1E0C09300010E94D32840
:105730000E94032AC093B7028EE00E943420BC016D
:1057400090E080E00E943F3960939402709395024C
:1057500080939602909397021092A9028091B102D1
:105760009091B20224E630E030939F0220939E0293
:1057700020E233E030939D0220939C022AE030E047
:1057800030939B0220939A02880F991F9093AB024B
:105790008093AA02CF91FF90EF90DF90CF90BF90BF
:1057A000AF909F908F90089520E030E040EA50EC59
:1057B000C701B6010E943A3987FF6CCF6091B302EE
:1057C0007091B4028091B5029091B6020E94EC3BB8
:1057D0007093C0026093BF025DCFC701B6019058BD
:1057E00077CF10924E0188CF0C945E3A2F923F9261
:1057F0004F925F926F927F928F929F92AF92BF92E1
:10580000CF92DF92EF92FF920F931F93CF93DF938C
:10581000CDB7DEB768970FB6F894DEBF0FBECDBF29
:1058200026E02093BF0721E02093BE071092BD071A
:105830000091AB071091AC076091A7077091A80782
:1058400030E8232E32E0332EF10130E020E0201743
:10585000310730F4DB01A20FB31F6115710521F48C
:1058600010927302A3E7B2E04C9150E04193519340
:105870002F5F3F4F2330310551F71C8A1B8A1E8A48
:105880001D8A188E1F8A4AE08E010F5F1F4FB801D4
:105890000E94F038F80101900020E9F73197AF013C
:1058A000401B510BB801CE0143960E94B029809154
:1058B000A7079091A807009709F4E8C06B897C8935
:1058C0006115710509F4E0C04091A9075091AA073C
:1058D0002F89388D4217530708F4D6C00E942B3EFB
:1058E0008F89988D9093AC078093AB07188E1F8A91
:1058F0008B899C89009711F00E94D73C94E7E92E90
:1059000092E0F92E24E0A22EB12CD12CC12C809152
:10591000AB079091AC07C816D90638F4E091A707F9
:10592000F091A807309709F0C8C010927302E3E71E
:10593000F2E0808190E0F10120813181821B930BA4
:10594000F2E3F89FB001F99F700D1124072E000CAF
:10595000880B990B0E944139F701208131814281E6
:1059600053810E94073B2B013C0120E030E0A9015C
:105970000E943A398111A4C0F701408251826282AB
:10598000738201E022E346E270E060E0C501049723
:105990000E94AB1A8EEC882E99249A940FEF1FEF79
:1059A000F701208131814281538160E070E080E81D
:1059B00090E40E94063B2B013C01B401092C000C31
:1059C000880B990B0E9441399B01AC01C301B201C4
:1059D0000E94073B0E94E53BB092BA07A092B9072C
:1059E0007093BC076093BB07F10160817181600F08
:1059F000711F60537109072E000C880B990B0E94D0
:105A000078260F5F1F4FF2E38F0E911C02301105B5
:105A100039F62FEFC21AD20A84E0E80EF11CECE24C
:105A2000AE0EB11CF2E02F0E311C23E0C216D104E1
:105A300009F06DCF00E022E040E870E060E090E027
:105A400080E00E94AB1A2DE040E863E370E090E054
:105A500080E00E94AB1A68960FB6F894DEBF0FBEC6
:105A6000CDBFDF91CF911F910F91FF90EF90DF900D
:105A7000CF90BF90AF909F908F907F906F905F90EE
:105A80004F903F902F9008950E94D73C8B899C891E
:105A90009093A8078093A7078D899E899093AA0762
:105AA0008093A9078F89988D9093AC078093AB075B
:105AB0001C8A1B8A1E8A1D8A19CFEC0DFD1D39CF49
:105AC000C301B20190582DEC3CEC4CE45FE30E9422
:105AD000A039A30192010E94073BF7016083718303
:105AE000828393834ECF86E00E94991C21E0892B0C
:105AF00009F020E0209399020E944F1B8091AA0296
:105B00009091AB02959587950E94F62B0E94031EFB
:105B10000E948A2086E00E94991C892B69F7809157
:105B200099028111E9CF0E949C208091A707909152
:105B3000A807009721F00E94C938CB01089560E0C2
:105B400070E0CB01FACF1F920F920FB60F92112483
:105B50002F933F934F935F936F937F938F939F9375
:105B6000AF93BF93EF93FF9382EC96E00E94E11B0B
:105B7000FF91EF91BF91AF919F918F917F916F9125
:105B80005F914F913F912F910F900FBE0F901F90FB
:105B900018951F920F920FB60F9211242F938F9387
:105BA0009F93EF93FF93E091D206F091D30680810B
:105BB000E091D806F091D90682FD1BC090818091BA
:105BC000DB068F5F8F732091DC06821741F0E09136
:105BD000DB06F0E0EE53F94F958F8093DB06FF91E3
:105BE000EF919F918F912F910F900FBE0F901F906B
:105BF00018958081F4CF1F920F920FB60F92112447
:105C00002F933F938F939F93AF93BF93809187027E
:105C100090918802A0918902B0918A023091860207
:105C200023E0230F2D3758F50196A11DB11D2093B8
:105C300086028093870290938802A0938902B09392
:105C40008A0280918B0290918C02A0918D02B0917A
:105C50008E020196A11DB11D80938B0290938C0240
:105C6000A0938D02B0938E02BF91AF919F918F91BF
:105C70003F912F910F900FBE0F901F90189526E81F
:105C8000230F0296A11DB11DD2CF1F920F920FB606
:105C90000F9211242F933F934F935F936F937F93B2
:105CA0008F939F93EF93FF9383B1817029B190916C
:105CB0009102981709F49DC030E0220F232F221F74
:105CC000330B922F8093910240919002241709F494
:105CD00090C02093900220919A0230919B029817D5
:105CE00019F03195219531094091AA025091AB02EA
:105CF00060919E0270919F02240F351F261737076F
:105D00000CF48BC020919A0230919B02981719F0E5
:105D10003195219531094091AA025091AB026091D1
:105D20009C0270919D02240F351F621773070CF4BB
:105D30006FC040919A0250919B02981719F05195AB
:105D4000419551092091AA023091AB02240F351FD1
:105D50003093AB022093AA0241E0981340E02091D7
:105D60008F02421709F440C020919A0230919B02A1
:105D7000981719F03195219531096091AA02709117
:105D8000AB02E0919E02F0919F02260F371F2E1763
:105D90003F070CF44CC020919A0230919B02981757
:105DA00019F03195219531096091AA027091AB02E9
:105DB000E0919C02F0919D02260F371FE217F30736
:105DC0008CF120919A0230919B02981719F031952D
:105DD000219531098091AA029091AB02820F931F05
:105DE0009093AB028093AA0240938F0281E080934C
:105DF000B702FF91EF919F918F917F916F915F918A
:105E00004F913F912F910F900FBE0F901F901895BB
:105E100020919C0230919D029BCF20919E02309157
:105E20009F0296CF80919C0290919D02D9CF809144
:105E30009E0290919F02D4CF18950F931F93CF93FA
:105E4000DF93E2ECF6E01382128288EE93E0A0E0AA
:105E5000B0E084839583A683B78388E492E091833E
:105E6000808385EC90E09587848784EC90E0978729
:105E7000868780EC90E0918B808B81EC90E0938B17
:105E8000828B82EC90E0958B848B86EC90E0978BF4
:105E9000868B118E128E138E148EEDEAF7E013822C
:105EA00012821682178280E1808715821482128600
:105EB0008AE592E09183808315861486178616867C
:105EC00011E0108B118A128B138AE7EAF7E0118236
:105ED0001082138212821582148250E040E060E743
:105EE00072E0CF010E94B029CBE6D7E083E697E0CD
:105EF0009F8F8E8F87E697E09D8F8C8F8FE597E041
:105F000099A388A31AAE1AAA1BAA1CAA1DAA80E0EC
:105F100090E0AFE7B3E48EAB9FABA8AFB9AF84E638
:105F200090E0A0E0B0E08EA79FA7A8ABB9AB81E05E
:105F300090E0998F888F9B8F8A8F1BAF80E090E0D5
:105F4000A0E3B1E488839983AA83BB8380E090E0D7
:105F5000A0E0BFE38C839D83AE83BF8380E090E0AD
:105F6000A0E8BFE388879987AA87BB8780E090E095
:105F7000A0E3B1EC8C879D87AE87BF878DEC9CEC4E
:105F8000ACE4BDEB888B998BAA8BBB8B80E090E057
:105F9000A0E2B1EC8C8B9D8BAE8BBF8B0E94DB1D86
:105FA0000EA51FA528A939A9601B710B820B930BA5
:105FB0006AA37BA38CA39DA3DF91CF911F910F9127
:105FC0000895CF93DF93CDB7DEB72A970FB6F89435
:105FD000DEBF0FBECDBF789484B5826084BD84B52A
:105FE000816084BD85B5826085BD85B5816085BDD4
:105FF00080916E00816080936E001092810080918C
:106000008100826080938100809181008160809313
:106010008100809180008160809380008091B10038
:1060200084608093B1008091B00081608093B00063
:1060300080917A00846080937A0080917A008260F7
:1060400080937A0080917A00816080937A008091B9
:106050007A00806880937A001092C1001092B90093
:1060600088E48093B8000E94F91D80E00E94EF1D33
:1060700001EA10E380ECE82E80E3F82EF801849129
:106080000E94EF1D0F5F1F4FE016F106B9F70E9447
:10609000E71D11E01093B8000E94031E81E2809377
:1060A000B50760E08EE00E94F01C60E08FE00E9487
:1060B000F01C61E085E00E94F01C61E089E00E9434
:1060C000F01C62E087E00E94F01C62E088E00E9421
:1060D000F01C62E086E00E94F01C62E08AE00E9410
:1060E000F01C8FEF90E00E942C1D60E085E00E9484
:1060F000C21C80917A00876080937A0080917A0038
:10610000886080937A00789410936B0010936800F5
:106110001BBB90E080E00E94F42B182F81E090E000
:106120000E94F42B912F8F30984009F0B5C082E087
:1061300090E00E94F42B182F83E090E00E94F42B53
:10614000912F909347018093460184E090E00E9454
:10615000F42B182F85E090E00E94F42B912F909360
:1061600045018093440186E090E00E94F42B8093E7
:10617000430187E090E00E94F42B80934C0188E07B
:1061800090E00E94F42B80934B0189E090E00E9404
:10619000F42B80934A018AE090E00E94F42B8093D4
:1061A000C1028BE090E00E94F42B91E0811101C0CC
:1061B00090E0909349018CE090E00E94F42B91E0F4
:1061C000811101C090E0909348018DE090E00E9421
:1061D000F42B8093BE028EE090E00E94F42B282ED8
:1061E000809342018FE090E00E94F42B8093BA02EA
:1061F00080E190E00E94F42B91E0811101C090E0D9
:1062000090939802A2E08A2EA1E09A2EBFE4AB2ED2
:10621000B1E0BB2E11E1E12EF12C312C231409F455
:1062200047C010E000E0C701800F911F0E94F42BCF
:10623000F501E00FF11F80830F5F1F4F063011053E
:1062400091F7670126E0C20ED11C3EE0E30EF11C7F
:106250003401C6010E94F42B082F10E0102F0027F4
:10626000F301118300832601F2E04F0E511CC60199
:1062700001960E94F42B082BF301019311933F0127
:1062800062014E145F0429F73394F8E08F0E911CDD
:1062900026E0A20EB11CC2CF68E090E080E00E9430
:1062A000EF296FE081E090E00E94EF290E94032A2D
:1062B0001091980280EC111101C088EC0E94201E00
:1062C00080EA111101C081EA0E94201E0E94BA1FBB
:1062D00090939302809392020E9462209093B9025D
:1062E0008093B80200914601109147011093B202C9
:1062F0000093B1028EE00E943420BC0190E080E067
:106300000E943F39609394027093950280939602A5
:10631000909397020E94F61F0E947C2520E030E0B7
:1063200040EA51E46091B3027091B4028091B502E9
:106330009091B6020E94073B6B017C01B80190E08E
:1063400080E00E943F399B01AC01C701B6010E9469
:106350003A3987FF04C090E080E00E942C1D109223
:106360009D0710929E0710929F071092A007412C44
:10637000512CEFE76E2EE3E47E2E4092A10750925F
:10638000A2076092A3077092A407A0908907B0901B
:106390008A078091A507F501C080D180E280F38053
:1063A000882309F4C1C6A3019201C701B6010E9466
:1063B0001B3C181634F5F5014082518262827382CB
:1063C0008090910790909207A0909307B0909407C7
:1063D000C090A107D090A207E090A307F090A40777
:1063E000A7019601C501B4010E941B3C1816C4F414
:1063F000C0929107D0929207E0929307F09294078F
:106400001FC020E030E0A901C701B6010E943A395F
:1064100087FFD6CFF5011082118212821382D0CF6E
:10642000C0909D07D0909E07E0909F07F090A00736
:10643000A7019601C501B4010E943A3987FDD8CF62
:1064400081E08093A50783B181708093910289B127
:1064500090E0880F892F881F990B809390022091DC
:1064600091029091900281E0291380E080938F0245
:1064700084E690E090939F0280939E0280E293E0F6
:1064800090939D0280939C028AE090E090939B02FF
:1064900080939A02000F111F1093AB020093AA027F
:1064A0000E94DB1D6093AD027093AE028093AF0239
:1064B0009093B0020E949C200E949C202090AA02EF
:1064C0003090AB029101359527953A872987309313
:1064D000B2022093B10286E00E94991C482E8111DD
:1064E0009EC08091A902882309F499C00E949C2033
:1064F0000E94DB1D6B017C01C092A502D092A60216
:10650000E092A702F092A80286E00E94991C892BD3
:1065100059F40E94DB1D6C197D098E099F09643FA7
:1065200071408105910580F30E94DB1D6C197D0986
:106530008E099F09643F71408105910508F43FC4AD
:106540008FEF90E00E942C1D0E949C20512C4AE06D
:10655000642E712C1092A002852D0E94A921582E24
:10656000F7E0F81708F438C0E82FF0E0E654FD4CE7
:106570000C94353CD4327C35F23558366636A0362C
:10658000AE36B83620E030E0A901C701B6010E945E
:106590003A3987FF55CF10929107109292071092C7
:1065A0009307109294074CCF3EE1632E712C81E04B
:1065B0008093A002852D0E94A921582E22E08217E7
:1065C00009F434C2281708F4E8C0882309F410C17C
:1065D00031E0831709F40FC10E94032A81E0809300
:1065E000B70229853A853093B2022093B10284E63E
:1065F00090E090939F0280939E0280E293E09093BC
:106600009D0280939C028AE090E090939B0280938D
:106610009A02C1018E7F9093AB028093AA024092AE
:10662000A9028091BB02882309F110914A0111232C
:10663000E9F00E94DB1DC090A102D090A202E09080
:10664000A302F090A4026C197D098E099F0928EE1F
:1066500033E040E050E00E94D53A211738F0109224
:10666000BB020E949C2081E080934D018091B70283
:106670008823E9F18091BC02882349F120E030E0D1
:1066800040EA51E46091B3027091B4028091B50286
:106690009091B6020E94073B6B017C016091B102B0
:1066A0007091B20290E080E00E943F399B01AC0102
:1066B000C701B6010E943A3987FF04C090E080E02C
:1066C0000E942C1D0E949C2081E080934D0110921D
:1066D000B7021092BC021092BD020E94DB1D6093B3
:1066E000AD027093AE028093AF029093B0020E940D
:1066F000DB1D0091AD021091AE022091AF023091EE
:10670000B002601B710B820B930B20E63AEE40E067
:1067100050E00E94D53A122F2093AC028091BC0227
:1067200081110BC080914C01882339F0281728F083
:1067300081E08093BC020E949C208091BD02811167
:106740000BC080914B01882339F0181728F081E0A5
:106750008093BD020E949C200E94B22A0E944F2377
:106760000E94DB1D8091B607362F381B832F909136
:10677000B707992309F439C33093B8071092B707C4
:1067800080E090E0892B09F499CE0E94CD1B8823EC
:1067900009F494CE0E94000091CE83E0581609F4CB
:1067A00048C194E0591218CF80914201883008F016
:1067B000FECE91E0980F909342018093BE020E941A
:1067C000BA20E091BE0228E0E29FF0011124EE5FC2
:1067D000FE4F88ED90E09183808324E331E03383A2
:1067E000228386E891E09583848377826682DFCE78
:1067F0000E94D328DCCE8E010F5F1F4F812C912C7D
:106800005401839498EEE92E93E0F92ECC24C3949E
:10681000D12CE091BE0224E0E29FF0011124C401DA
:106820000197E80FF91FEE0FFF1FEE5FFE4F80810B
:1068300091819093B2028093B102E8ECF0E0F09382
:106840009F02E0939E02F0929D02E0929C02D09201
:106850009B02C0929A02880F991F9093AB0280937B
:10686000AA02F1E0F0934D0186E00E94991C21E01C
:10687000892B09F020E0209399020E944F1B22E00F
:106880002093BF070E94B22A0E944F231092BA079A
:106890001092B9071092BC071092BB0786EE90E3E6
:1068A0000E94971FC501B4010E9478268EE692E0EF
:1068B0000E94272680914E011092BA071092B907C4
:1068C000882309F48BC080E190E09093BC0780930B
:1068D000BB0789ED90E30E94971F1092BA071092B0
:1068E000B907E0E2F0E0F093BC07E093BB0782ED6C
:1068F00090E30E94971F6091AA027091AB02759578
:106900006795072E000C880B990B0E9478260E9431
:106910008A200E94031E86E00E94991C892B09F0A0
:10692000ACCF809199028111A8CF8091AA02909159
:10693000AB0295958795F801819391938F010E9401
:106940009C206AE070E080E090E00E94A91DFFEFCB
:106950008F1A9F0AAF0ABF0A24E082169104A1048D
:10696000B10409F056CF8FEF90E00E942C1D8BEA06
:1069700094E00197F1F70E94F61F0E94EC3B4B0157
:1069800078876F83C980DA800B811C81C6014E969F
:106990008017910708F00BCEED80FE80C8014E965F
:1069A0008E159F0508F003CE87E08093A00280E05B
:1069B0000E94A921882309F4FACDE091BE0238E0B3
:1069C000E39FF0011124EE5FFE4FD182C08213835A
:1069D0000283F582E48297828682E9CD20E130E06D
:1069E0003093BC072093BB078CEC90E30E94971F69
:1069F0006091940270919502809196029091970215
:106A00000E94EC3B90E080E04AE00E943426109225
:106A1000BA071092B90780E290E09093BC07809388
:106A2000BB0780EC90E30E94971F71CF0E94BA20B1
:106A3000BECD87E08093A00280914201813009F4AD
:106A4000B6CD80E00E94A921882309F4B0CD109131
:106A5000BE0200914201802F8150990BBC01181792
:106A6000190639F411501093BE02015000934201EF
:106A70009ECD812F90E086179707BCF7E6E01E9F1A
:106A8000D001112450E040E09C012F5F3F4FFA01FC
:106A9000EA0FFB1FE15BFE4FF680F0824F5F5F4F16
:106AA00046305105A1F743E0220F331F4A95E1F725
:106AB000F901EE5FFE4F2081318153E0880F991F6D
:106AC0005A95E1F7DC01AE5FBE4F11963C932E93D1
:106AD0008281938113969C938E93129784819581E2
:106AE00015969C938E9314978681978117969C9305
:106AF0008E9316971F5FBDCF82E08093A00210E0B7
:106B000008E2C02ED12C84E6A82EB12C90E2892E6A
:106B100093E0992E24E1E22EF12C812F0E94A921ED
:106B2000182F813021F130F0823009F43FC00E94EB
:106B3000032A10CD8091460190914701B0929F02A7
:106B4000A0929E0290929D0280929C0270929B0263
:106B500060929A02880F991F9093AB028093AA02C9
:106B60000E94732D9093470180934601D6CF809168
:106B7000440190914501D0929F02C0929E02E0E9AB
:106B8000F1E0F0939D02E0939C0270929B02609270
:106B90009A02880F991F9093AB028093AA020E94D9
:106BA000732D9093450180934401B7CF80914301A9
:106BB00090E0F0929F02E0929E0228EC30E0309349
:106BC0009D0220939C0270929B0260929A02880F11
:106BD000991F9093AB028093AA020E94732D809319
:106BE00043019BCF83E08093A00210E0812F0E949D
:106BF000A921182F8130F1F1F8F0823009F097CFF8
:106C000080914A0190E010929F0210929E02E8E665
:106C1000F1E0F0939D02E0939C0270929B026092DF
:106C20009A02880F991F9093AB028093AA020E9448
:106C3000732D80934A01DACF80914C0190E010923D
:106C40009F0210929E02ECE3F0E0F0939D02E0932D
:106C50009C0221E030E030939B0220939A02880F3F
:106C6000991F9093AB028093AA020E94732D809388
:106C70004C01BCCF80914B0190E010929F0210928A
:106C80009E02E8E7F0E0F0939D02E0939C0225E08D
:106C900030E030939B0220939A02880F991F9093C3
:106CA000AB028093AA020E94732D80934B019ECF6A
:106CB00084E08093A002809149010E94A92191E083
:106CC000811101C090E09093490144CC10E03AE07A
:106CD000E32E45E0D42E59E0C52EE092A002812F8C
:106CE0000E94A921182F882321F08130E1F000E0D3
:106CF00009C0D092A0028091C1020E94A921809374
:106D0000C10201E0F090980280ECF11001C088EC23
:106D10000E94201E80EAF11001C081EA0E94201E1C
:106D20000111DBCF04CFC092A002809198020E9493
:106D3000A92191E0811101C090E090939802E1CFE8
:106D400086E08093A002809148010E94A92191E0F1
:106D5000811101C090E090934801FCCB88E08093C2
:106D6000A0028091BA020E94A9218093BA02F2CBBC
:106D700086E00E94991C21E0892B09F020E02093F5
:106D800099020E944F1BEE24E39400E320E34DEEB2
:106D900050E368E070E088E290E00E94CD1A0E9423
:106DA000031E0E948A2086E00E94991C892BC9F745
:106DB000809199028111F5CF0E949C20CBCB8091CC
:106DC000BB0291E089278093BB02882351F00E9487
:106DD000DB1D6093A1027093A2028093A3029093A3
:106DE000A40281E08093B7021ACC9091B5073917BD
:106DF00048F48F5F891708F0C3CC81E083BF889582
:106E000013BEBECC11E01093B7076093B607809114
:106E1000B1079091B20701969093B2078093B107A2
:106E20008091C102882309F466C10E944F1B01E0D2
:106E300020E440E870E060E090E080E00E94AB1A5F
:106E40001093BF071093BE071092BD07E12C00E11D
:106E500020E144E852E370E060E090E080E00E94CE
:106E6000CD1A83E190E09093BA078093B90784E04C
:106E700090E09093BC078093BB078091BE02E6E050
:106E80008E9FC0011124815B9E4F0E942726809116
:106E9000BF029091C002853F914008F0F7C08091F9
:106EA000BD028111F5C08091BC028111F3C08091B7
:106EB000BB028111F1C080914E018111EFC020E031
:106EC00030E044E353E4609163077091640780917C
:106ED0006507909166070E943A3987FFE1C085E017
:106EE00025E330E03093BA072093B90721E030E082
:106EF0003093BC072093BB0792E09093BF07C82E46
:106F0000D12C9091BA02CC0CDD1C9111CBC0F601B2
:106F1000EA5CFD4F40815181E12C0EE02CE161E003
:106F200070E080E590E00E94CD1AF601E85DFD4F2B
:106F300040815181E12C00E120E170E060E080E7D8
:106F400090E00E94CD1A81E08093BF0720E14EE3DC
:106F500052E360E170E090E080E00E94CD1A20E111
:106F60004EE152E360E270E090E080E00E94CD1AD2
:106F700003E110E01093BA070093B90720E130E075
:106F80003093BC072093BB070E94F61F41E00E948C
:106F9000A22688EF0E94B21F8CE192E30E94971F05
:106FA0001093BA070093B90788E190E09093BC076B
:106FB0008093BB070E94BA1FBC0190E080E00E9452
:106FC0003F3920E030E04AE754E40E94733B42E05E
:106FD0000E94A2268AE192E30E94971F1093BA07AB
:106FE0000093B90780E290E09093BC078093BB07C1
:106FF0006091B8027091B90290E080E00E943F3940
:1070000020E030E04AE754E40E94733B41E00E94F4
:10701000A22688E192E30E94971F1093BA0700937B
:10702000B90788E290E09093BC078093BB0781E1A9
:1070300092E30E94971F89E390E09093BA078093B0
:10704000B90782E190E09093BC078093BB0784E08E
:107050008093BF076091BF027091C002653F91E0CD
:10706000790708F442C08DE092E30E94971F00E088
:1070700020E248E460E170E087E390E00E94641E53
:1070800080E00E947A270E94031E7ACB80E028CFFE
:1070900081E026CF82E024CF83E022CF84E020CF9E
:1070A00086E01ECF8330C1F038F4813069F0823041
:1070B00081F08EE592E30AC08530A1F080F0863041
:1070C000C1F784E692E302C080E892E30E94971F32
:1070D0002CCF8AE792E3FACF84E792E3F7CF8EE6EC
:1070E00092E3F4CF89E692E3F1CF90E080E04AE0CA
:1070F0000E943426BCCF0E944F1B8091BF0290910A
:10710000C002853FE1E09E0710F087EE93E00E9409
:10711000F62B00E023E040E860E370E090E080E0E0
:107120000E94AB1A81E0ADCFC0929107D092920736
:10713000E0929307F0929407E0918707F091880717
:1071400080819181A281B381809395079093960766
:10715000A0939707B093980720E030E04FE753E4FF
:10716000C701B6010E941B3C18160CF00BCA4092D6
:10717000910750929207609293077092940760C9AA
:107180008091A7079091A807009711F00C94D73C25
:1071900008951F93FC0199278827BC01E894119159
:1071A0001032E9F3193010F01E30C8F31B3251F0E1
:1071B0001D3249F4689406C00E94FB38610F711DAE
:1071C000811D911D119110531A30B0F33EF490952A
:1071D0008095709561957F4F8F4F9F4F1F910895B8
:1071E000BB274A3031F4992322F4BDE29095819572
:1071F0009F4F0C941139592F482F372F262F660F88
:10720000771F881F991F660F771F881F991F620FAE
:10721000731F841F951F660F771F881F991F08957E
:10722000BB27FB015527AA27880F991FAA1FA41760
:1072300010F0A41B83955051B9F7A05DAA3308F054
:10724000A95DA193009779F7B111B1931192CB0188
:107250000C942A39DC01FC01672F71917723E1F747
:10726000329704C07C916D9370836291AE17BF0713
:10727000C8F308950E947C3908F481E00895E894E9
:1072800009C097FB3EF490958095709561957F4F6E
:107290008F4F9F4F9923A9F0F92F96E9BB2793951C
:1072A000F695879577956795B795F111F8CFFAF42C
:1072B000BB0F11F460FF1BC06F5F7F4F8F4F9F4F5D
:1072C00016C0882311F096E911C0772321F09EE8BB
:1072D000872F762F05C0662371F096E8862F70E021
:1072E00060E02AF09A95660F771F881FDAF7880FFB
:1072F0009695879597F90895990F0008550FAA0B51
:10730000E0E8FEEF16161706E807F907C0F01216B8
:107310001306E407F50798F0621B730B840B950BBB
:1073200039F40A2661F0232B242B252B21F4089510
:107330000A2609F4A140A6958FEF811D811D0895AD
:107340000E94B3390C94243A0E94163A38F00E94F5
:107350001D3A20F0952311F00C940D3A0C94133A39
:1073600011240C94583A0E94353A70F3959FC1F35A
:10737000950F50E0551F629FF001729FBB27F00DE3
:10738000B11D639FAA27F00DB11DAA1F649F662738
:10739000B00DA11D661F829F2227B00DA11D621F87
:1073A000739FB00DA11D621F839FA00D611D221F41
:1073B000749F3327A00D611D231F849F600D211D25
:1073C000822F762F6A2F11249F5750409AF0F1F0A8
:1073D00088234AF0EE0FFF1FBB1F661F771F881F11
:1073E00091505040A9F79E3F510580F00C940D3A02
:1073F0000C94583A5F3FE4F3983ED4F38695779522
:107400006795B795F795E7959F5FC1F7FE2B880FB6
:10741000911D9695879597F9089597F99F6780E84C
:1074200070E060E008959FEF80EC089500240A94D6
:107430001616170618060906089500240A9412164F
:107440001306140605060895092E0394000C11F482
:10745000882352F0BB0F40F4BF2B11F460FF04C02F
:107460006F5F7F4F8F4F9F4F089557FD9058440F88
:10747000551F59F05F3F71F04795880F97FB991F93
:1074800061F09F3F79F08795089512161306140650
:10749000551FF2CF4695F1DF08C0161617061806DD
:1074A000991FF1CF86957105610508940895E894B8
:1074B000BB2766277727CB0197F90895F999FECF67
:1074C00092BD81BDF89A992780B50895262FF99924
:1074D000FECF1FBA92BD81BD20BD0FB6F894FA9AB7
:1074E000F99A0FBE01960895052E97FB1EF400949D
:1074F0000E948B3A57FD07D00E94D53A07FC03D073
:107500004EF40C948B3A50954095309521953F4F11
:107510004F4F5F4F089590958095709561957F4F7F
:107520008F4F9F4F08950E94F73AA59F900DB49FEB
:10753000900DA49F800D911D112408952F923F92CC
:107540004F925F926F927F928F929F92AF92BF9273
:10755000CF92DF92EF92FF920F931F93CF93DF931F
:10756000CDB7DEB7CA1BDB0B0FB6F894DEBF0FBE7C
:10757000CDBF09942A88398848885F846E847D84C9
:107580008C849B84AA84B984C884DF80EE80FD80CB
:107590000C811B81AA81B981CE0FD11D0FB6F89441
:1075A000DEBF0FBECDBFED010895A1E21A2EAA1BCA
:1075B000BB1BFD010DC0AA1FBB1FEE1FFF1FA217A3
:1075C000B307E407F50720F0A21BB30BE40BF50BA0
:1075D000661F771F881F991F1A9469F76095709529
:1075E000809590959B01AC01BD01CF010895A29FAC
:1075F000B001B39FC001A39F700D811D1124911D87
:10760000B29F700D811D1124911D08955058BB2704
:10761000AA270E941E3B0C94243A0E94163A38F086
:107620000E941D3A20F039F49F3F19F426F40C947F
:10763000133A0EF4E095E7FB0C940D3AE92F0E9403
:10764000353A58F3BA17620773078407950720F095
:1076500079F4A6F50C94573A0EF4E0950B2EBA2F58
:10766000A02D0B01B90190010C01CA01A001112448
:10767000FF27591B99F0593F50F4503E68F11A16F4
:10768000F040A22F232F342F4427585FF3CF469585
:1076900037952795A795F0405395C9F77EF41F16A7
:1076A000BA0B620B730B840BBAF09150A1F0FF0F71
:1076B000BB1F661F771F881FC2F70EC0BA0F621F5D
:1076C000731F841F48F4879577956795B795F7954D
:1076D0009E3F08F0B0CF9395880F08F09927EE0FE2
:1076E0009795879508950E94873B0C94243A0E94B1
:1076F0001D3A58F00E94163A40F029F45F3F29F0F5
:107700000C940D3A51110C94583A0C94133A0E946F
:10771000353A68F39923B1F3552391F3951B550B33
:10772000BB27AA2762177307840738F09F5F5F4F54
:10773000220F331F441FAA1FA9F335D00E2E3AF093
:10774000E0E832D091505040E695001CCAF72BD0AB
:10775000FE2F29D0660F771F881FBB1F26173707FC
:107760004807AB07B0E809F0BB0B802DBF01FF272E
:1077700093585F4F3AF09E3F510578F00C940D3AC4
:107780000C94583A5F3FE4F3983ED4F3869577958E
:107790006795B795F7959F5FC9F7880F911D9695E7
:1077A000879597F90895E1E0660F771F881FBB1F43
:1077B000621773078407BA0720F0621B730B840BF0
:1077C000BA0BEE1F88F7E09508950E94EC3B689491
:1077D000B1110C94583A08950E943D3A88F09F5791
:1077E00098F0B92F9927B751B0F0E1F0660F771FE5
:1077F000881F991F1AF0BA95C9F714C0B13091F0DB
:107800000E94573AB1E008950C94573A672F782FA9
:107810008827B85F39F0B93FCCF38695779567959F
:10782000B395D9F73EF490958095709561957F4F0B
:107830008F4F9F4F08950E947C3908F48FEF089571
:107840000E947C39880B990B0895DB018F939F93DD
:107850000E94933ABF91AF91A29F800D911DA39F6B
:10786000900DB29F900D11240895EE0FFF1F05900B
:10787000F491E02D09940F931F93CF93DF938230FF
:10788000910510F482E090E0E091C307F091C40705
:1078900030E020E0B0E0A0E0309799F42115310508
:1078A00009F44AC0281B390B24303105D8F58A81E8
:1078B0009B816115710589F1FB0193838283FE0130
:1078C00011C0408151810281138148175907E0F0AE
:1078D0004817590799F4109761F012960C93129774
:1078E00013961C933296CF01DF91CF911F910F9188
:1078F00008950093C3071093C407F4CF21153105F1
:1079000051F04217530738F0A901DB019A01BD017C
:10791000DF01F801C1CFEF01F9CF9093C407809345
:10792000C307CDCFFE01E20FF31F81939193225045
:10793000310939832883D7CF2091C1073091C207FD
:10794000232B41F420918101309182013093C207B1
:107950002093C10720917F013091800121153105CD
:1079600041F42DB73EB74091830150918401241B0F
:10797000350BE091C107F091C207E217F307A0F4BD
:107980002E1B3F0B2817390778F0AC014E5F5F4F75
:107990002417350748F04E0F5F1F5093C2074093DE
:1079A000C107819391939FCFF0E0E0E09CCFCF930C
:1079B000DF930097E9F0FC01329713821282A091C5
:1079C000C307B091C407ED0130E020E01097A1F4A7
:1079D00020813181820F931F2091C1073091C2070E
:1079E0002817390709F061C0F093C207E093C10777
:1079F000DF91CF910895EA01CE17DF07E8F54A81BC
:107A00005B819E0141155105B1F7E901FB83EA83D2
:107A100049915991C40FD51FEC17FD0761F480817E
:107A200091810296840F951FE90199838883828151
:107A300093819B838A83F0E0E0E012968D919C9184
:107A400013970097B9F52D913C911197CD010296AE
:107A5000820F931F2091C1073091C2072817390761
:107A600039F6309751F51092C4071092C307B093BE
:107A7000C207A093C107BCCFD383C2834081518189
:107A8000840F951FC817D90761F44E5F5F4F888137
:107A90009981480F591F518340838A819B81938329
:107AA00082832115310509F0B0CFF093C407E0932C
:107AB000C3079ECFFD01DC01C0CF13821282D7CF56
:107AC000B0E0A0E0E6E6FDE30C94A03A8C0100975C
:107AD00051F4CB010E943B3C8C01C801CDB7DEB70D
:107AE000E0E10C94BC3AFC01E60FF71F9C01225028
:107AF0003109E217F30708F49DC0D901CD91DC915B
:107B00001197C617D70798F0C530D10530F3CE01CD
:107B100004978617970708F3C61BD70B2297C193C4
:107B2000D1936D937C93CF010E94D73CD6CF5B015C
:107B3000AC1ABD0A4C018C0E9D1EA091C307B091DA
:107B4000C407512C412CF12CE12C109731F5809178
:107B5000C1079091C2078815990509F05CC04616C7
:107B6000570608F058C080917F01909180010097DE
:107B700041F48DB79EB74091830150918401841BDD
:107B8000950BE817F90708F055C0F093C207E0938A
:107B9000C107F90171836083A0CF8D919C911197EA
:107BA00012966C90129713967C901397A815B905AE
:107BB00059F56C0142E0C40ED11CCA14DB0420F15B
:107BC000AC014A195B09DA011296159780F06282BE
:107BD000738251834083D9016D937C93E114F10446
:107BE00071F0D7011396FC93EE93129776CF2296FD
:107BF0008C0F9D1FF90191838083F301EFCFF093E8
:107C0000C407E093C30769CF4816590608F42C014E
:107C10007D01D3019ACFCB010E943B3C7C010097B0
:107C200049F0AE01B8010E94223EC8010E94D73C33
:107C3000870153CF10E000E050CF81E090E0F8944E
:107C40000C94323EFB01DC0102C001900D924150C8
:107C50005040D8F70895FB01DC0101900D920020FF
:107C6000E1F7089519E1C1E6D9E104C0FE010E94DF
:107C7000353C2196C236D107C9F7F894FFCF01FFF2
:107C8000D800340186011E00000000000000000042
:107C900000000000000000000000000000000000E4
:107CA00000000000000000000000000000000000D4
:107CB00000000000000000000000000000000000C4
:107CC000013C960040010101280F050101424331AA
:107CD0002E35000000000000000000000000000041
:107CE0000000000000000000000000000000000094
:107CF000000000000000000000000000000000C5BF
:107D000007800078092809D80888083808E8079803
:107D1000074807F8067809A80658060806B805684F
:107D2000051805C80478046805C8042804780468A0
:107D300005D80388033803E80298024802F801A82E
:107D40000158010801F801A801B800680068050899
:107D500027E825C824A823882268214820281F084E
:107D60001EE81CC81B0827A81A8819681808274885
:107D700017281668184817081528166818E813C831
:107D800012A8118810680F6821480E280D080CE809
:107D90000A480E280DA811C809681809060404022B
:107DA000020202020203C828A82888281E32682876
:107DB00048282828382A002AC82990295829202903
:107DC000E82800000000031C631B901B501CC11B13
:107DD0009F1BB31B00000000951E631BB71F621B97
:107DE0006E616E00696E66006F7666002F3300006C
:107E0000112484B714BE81FFF0D085E080938100F7
:107E100082E08093C00088E18093C10086E0809377
:107E2000C20080E18093C4008EE0C9D0259A86E02C
:107E300020E33CEF91E0309385002093840096BBD3
:107E4000B09BFECF1D9AA8958150A9F7CC24DD24C4
:107E500088248394B5E0AB2EA1E19A2EF3E0BF2EE7
:107E6000A2D0813461F49FD0082FAFD0023811F036
:107E7000013811F484E001C083E08DD089C08234E0
:107E800011F484E103C0853419F485E0A6D080C0E4
:107E9000853579F488D0E82EFF2485D0082F10E0AE
:107EA000102F00270E291F29000F111F8ED06801E7
:107EB0006FC0863521F484E090D080E0DECF843638
:107EC00009F040C070D06FD0082F6DD080E0C81688
:107ED00080E7D80618F4F601B7BEE895C0E0D1E017
:107EE00062D089930C17E1F7F0E0CF16F0E7DF06D8
:107EF00018F0F601B7BEE89568D007B600FCFDCFD4
:107F0000A601A0E0B1E02C9130E011968C91119780
:107F100090E0982F8827822B932B1296FA010C0160
:107F200087BEE89511244E5F5F4FF1E0A038BF0790
:107F300051F7F601A7BEE89507B600FCFDCF97BE46
:107F4000E89526C08437B1F42ED02DD0F82E2BD052
:107F50003CD0F601EF2C8F010F5F1F4F84911BD097
:107F6000EA94F801C1F70894C11CD11CFA94CF0C13
:107F7000D11C0EC0853739F428D08EE10CD085E9AC
:107F80000AD08FE07ACF813511F488E018D01DD067
:107F900080E101D065CF982F8091C00085FFFCCF94
:107FA0009093C60008958091C00087FFFCCF809118
:107FB000C00084FD01C0A8958091C6000895E0E648
:107FC000F0E098E1908380830895EDDF803219F02E
:107FD00088E0F5DFFFCF84E1DECF1F93182FE3DFCA
:107FE0001150E9F7F2DF1F91089580E0E8DFEE27F6
:047FF000FF270994CA
:027FFE00040479
:00000001FF
